S31508001800A00A0020D9180008E7180008E9180008F7
S3150800181000000000000000000000000000000000BA
S315080018200000000000000000000000000119000888
S31508001830000000000000000003190008593B0008DA
S31508001840B94B000807190008071900080719000806
S3150800185007190008071900080719000807190008DA
S31508001860071900089D290008071900080719000824
S3150800187007190008071900080719000807190008BA
S3150800188007190008000000000000000007190008FA
S3150800189000000000071900080719000807190008C2
S315080018A0000000000719000807190008E1450008AC
S315080018B007190008071900080719000800000000A2
S315080018C0EE11AA550348854600F006FD0048004774
S315080018D02D750008A00A00200B4880F308880B48DD
S315080018E080470B480047FEE704207146084202D0AD
S315080018F0EFF3098001E0EFF30880714605F082FCFA
S31508001900FEE7FEE7FEE7FEE7A00A0020C13D000865
S31508001910C518000830B50B460146002020220124D0
S3150800192009E00D46D5409D4205D31D469540491B05
S315080019302546954040191546521E002DF1DC30BD4E
S3150800194070B500242546002801DA01244042002902
S3150800195001DA01254942FFF7DDFFAC4200D04042DB
S31508001960002C00D0494270BD03460B439B0703D0A9
S3150800197009E008C9121F08C0042AFAD203E00B7846
S315080019800370401C491C521EF9D27047D2B201E0BE
S315080019900270401C491EFBD270470022F6E710B5BC
S315080019A013460A4604461946FFF7F0FF204610BDBF
S315080019B0F8B502464A40D40F42004B0052085B086D
S315080019C09A4202D20246084611464A0023D0C30D5F
S315080019D04A00DDB2120EAD1A202D35DA490201266B
S315080019E0490AF6058A19002C00D0524220214F1BBD
S315080019F01146B9402A411018C20D9A4221D0002C2E
S31508001A0017D0012D08DCDA05801AD20F8019D20703
S31508001A10DBB200F077FBF8BDDA05801A0123400037
S31508001A201B06C01880185A428018CA0F104349006E
S31508001A3007E04908C2071143DA05801A80194008E9
S31508001A40801800F057FBF8BD61000122511A001BEF
S31508001A50F7E70122D2075140AAE70122D2075040F0
S31508001A60A6E7024670B54A40D30FDB0740002DD0E3
S31508001A704A002AD0010E140E000212020919400A61
S31508001A80520A8418E50104465443000A120A2E0431
S31508001A905043A4194219200CC543AA18120C012553
S31508001AA0AD03521C521912047F39240400D0521C6B
S31508001AB0104301D44000491EC2B20C06C0092018C2
S31508001AC0401C4008802A02D003E0002070BD400870
S31508001AD04000002900DA0020184370BD70B50246A0
S31508001AE04A40D50F40004A00ED0740085208002832
S31508001AF014D0002A12D0C40DD30D41020120C0050E
S31508001B005202490A520AE41A091812187D349142F7
S31508001B1001D3641C00E04900002C01DA002070BDE6
S31508001B200023914201D3891A03434008490000283B
S31508001B30F7D100290AD0914202D10121C90705E04F
S31508001B40914201D2012101E00121C943E005C018F3
S31508001B50401900F0CFFA70BDF0B507460846584060
S31508001B6087B0C00F049048000E465900400849083F
S31508001B70BC1A884105D2384631461E4617460B46DA
S31508001B8002465800400810434CD0300D03904005DB
S31508001B905900400D490D0590401A0290402872DA06
S31508001BA018030121000B09050843019004980092C7
S31508001BB0002805D0019952420020884100920190E0
S31508001BC0029840210A1A0199009800F05FFA054622
S31508001BD00C466B4607CB00F07AFAC0197141039A96
S31508001BE00E0D0023D71756401A467A40164344D09E
S31508001BF0049A002A2DD0029A012A039A15DC1205A6
S31508001C00C01A914101263605001C7141D20F059E66
S31508001C10D2070093019202962A46234600F0B8FAA4
S31508001C2007B0F0BD38463146FAE71605224A0F4690
S31508001C30B218C01AB74101210905001C4F41001806
S31508001C407F41114618187941E20F10436D19644116
S31508001C5013E0E2076D0815436408C2071443039AA4
S31508001C6001261205C01A91413605001C7141CE079E
S31508001C70400830434908C01851412A46234600F017
S31508001C807AFACDE7FFE7049801224000C117121A35
S31508001C9000238B4104983146C417381AA141EEE750
S31508001CA030B40124E407634030BC55E730B401245E
S31508001CB0E407614030BC4FE70000E0FFF0B51FB411
S31508001CC088B00B990998002448400999C00F490023
S31508001CD049080991C0070B990090490049080B91DA
S31508001CE009990898A64608431CD00B990A980843F0
S31508001CF018D0099801244000420D4800410D099862
S31508001D0024050003000B204309900B980003000BE1
S31508001D1020430B9050181C49401800220190144685
S31508001D20104605E0002001460DB0F0BD032801DA93
S31508001D30034600E003239C46C11A0AAE0AE05F0088
S31508001D4008ADED5B4F00F75B7D430027AA187C4181
S31508001D50491C5B1E6145F2DD410004AB5A52210461
S31508001D60120C0A43240C401C0828DFDB0198029059
S31508001D700099704601910090059B049A0799069868
S31508001D8000F006FAD0E700000DFCFFFFF0B50C46A0
S31508001D905C4085B0E40FE40703944C000026640811
S31508001DA059009446490802460296224321D06246C3
S31508001DB00A431ED06200570D4A000E032303550D31
S31508001DC0012402462C492405781B1B0B360B4018A8
S31508001DD023432643614600901C46501AB44103D358
S31508001DE00098401C009002E0921800985B41002879
S31508001DF003DA0020014605B0F0BD002001210905DF
S31508001E000746864611E064461D46141BB54106D3AF
S31508001E106546521BB341744607430C43A646CD0795
S31508001E2040084908284392185B4105460D43EAD104
S31508001E301046184313D0604619465040714008436F
S31508001E4006D06046101AB34106D20122002306E0E6
S31508001E5000220123DB0702E00122D2435310009837
S31508001E6074460105381C6141029C039D00196941AD
S31508001E7000F081F9BFE70000FD030000C217C10F9B
S31508001E80504010B54018CA079623002100F03AF9C9
S31508001E9010BD10B500229623114600F033F910BD87
S31508001EA00EB5C217C10F5040CA0740180021054B8E
S31508001EB00293019200910A460B4600F069F903B0B5
S31508001EC000BD0000330400000EB50549029100214B
S31508001ED000910A460B46019100F05AF903B000BD7D
S31508001EE033040000C20F410040020123400ADB050B
S31508001EF0D207090EC0187F2901DA002070479629F3
S31508001F0003DC9623591AC84001E096398840002A0E
S31508001F10F4D040427047410040020122400AD205EF
S31508001F20090E80187F2901DA00207047962903DCFC
S31508001F309622511AC8407047963988407047000063
S31508001F404A0009030123090B1B051943094B10B560
S31508001F50520D9A4201DA002010BD064B34339A42DC
S31508001F6003DC9A1A00F0A2F810BD034951188840FC
S31508001F7010BD0000FF030000CDFBFFFFC20FD20714
S31508001F80400040080BD0C10D0723DB01C9184002E9
S31508001F900905400A1143C20840071143704700204B
S31508001FA00146704710B5002904DB0124E4074042C6
S31508001FB08C412146002B04DB1C460123DB075242D9
S31508001FC0A3418B4200D1824210BD0000CB0FDB0734
S31508001FD0490010B5490802460A4307D00A0D0724E6
S31508001FE00903E401090B121B002A01DC002010BDBD
S31508001FF0C900440F0C43C100E018D205801800F050
S3150800200079F810BD0122D207002800DB101A002932
S3150800201000DB511A814270470122D207002800DBF3
S31508002020101A002900DB511A88427047F0B51FB410
S315080020300646002082B005464024019100901BE028
S31508002040019922460F46304600F030F8049A059B5F
S31508002050801A994110D310461946224600F016F800
S31508002060361A8F410197224601200021009F00F071
S315080020700DF838184D4100902046641E0028DFDC14
S31508002080019B00982946324607B0F0BD10B5202AB4
S3150800209004DB0146203A9140002010BD91402023E0
S315080020A09C1A0346E3401943904010BD10B5202AF8
S315080020B004DB0846203AD040002110BD0B46D34029
S315080020C0D0402024A21A91400843194610BD10B5E5
S315080020D0202A06DBCB170846203A1041C1170B43C6
S315080020E006E00B461341D0402024A21A914008432B
S315080020F0194610BD002904DA401C490001D14008E0
S315080021004000704770B40024050C05D11024000463
S3150800211002D1002921D01124050E01D1000208346C
S31508002120050F01D10001241D850F01D18000A41CD3
S31508002130002801DB4000641C002908D020252E1B3E
S315080021400D46F540A14000D0012129430843010668
S315080021501B1B000ADB1D02D5002070BC7047DB057F
S31508002160181880180029F8DA401C4900F5D170BC07
S3150800217040084000704710B5002B08DA0024401CC0
S31508002180614192185B411A4301D14008400010BDD5
S31508002190F0B51FB482B005460C0003D0084602F01D
S315080021A077FD02E002F074FD2030024600902146D9
S315080021B02846FFF76BFF049B059A04460F4618430B
S315080021C01143084314D0184610431BD000984021E9
S315080021D00A1A18460599FFF769FF05460E46009A3A
S315080021E005990498FFF752FF084305D0012004E03B
S315080021F02046394607B0F0BD0020C11705430E43F7
S315080022002C43374300990E986305401A7905E40A6A
S3150800221000220C43FD0A0A3002D500200146E9E7F0
S315080022200105101969410C9C0D9D00196941FFF7BC
S31508002230A2FFDFE7FEB500231A461B1A8A4103DB15
S315080022400020014603B0F0BD4A000D0301212D0B05
S315080022500905520D0D43D10702D100186D41521ED2
S315080022605110FF31FF310131002704463E463846FA
S31508002270009701910246012100200905FFF716FF84
S31508002280C3197141F818324684468E464A4161465A
S315080022902846611A904104D36046241A9541764629
S315080022A01F46241900986D41401C00903428E1DD32
S315080022B0F91930467041091BA84103D20022D243BE
S315080022C0134601E00022134601980105381C7141A6
S315080022D0FFF751FFB6E70000064C0125064E05E05C
S315080022E0E36807CC2B430C3C98471034B442F7D329
S315080022F0FFF7ECFA94910008B491000870B58C18B1
S315080023000578401C6B075B0F01D10378401C2A1126
S3150800231006D10278401C03E006780E70401C491C62
S315080023205B1EF9D12B0705D40023521E0DD40B7062
S31508002330491CFAE70378401CCB1A921C03E01D7867
S315080023400D70491C5B1C521EF9D5A142D8D300203A
S3150800235070BD000010B50446002C08D101210920E3
S31508002360C00600F0E7FD002000F0E6F852E0012C78
S3150800237005D102210920C00600F0DCFD4AE0022C46
S3150800238005D104210920C00600F0D4FD42E0032C43
S3150800239005D108210920C00600F0CCFD3AE0042C3E
S315080023A005D110210920C00600F0C4FD32E0052C35
S315080023B005D120210920C00600F0BCFD2AE0062C24
S315080023C005D140210920C00600F0B4FD22E0072C03
S315080023D005D180210920C00600F0ACFD1AE0082CC2
S315080023E004D101210D4800F0A5FD13E0092C04D104
S315080023F002210A4800F09EFD0CE00B2C04D11021A6
S31508002400064800F097FD05E00C2C03D1802103480F
S3150800241000F090FD204600F08FF810BD000400483B
S315080024207FB500200090019002900390002427E0D9
S3150800243000250CE0E800294940186100405AA1002F
S315080024406A4651584018A1005050681C85B2142D90
S31508002450F0DBA1006A4650581421FFF75BFA2821E1
S31508002460484361001E4A515A3C225143461864218A
S315080024703046FFF74FFA6100194A5052601C84B281
S31508002480042CD5DB1748407B002826D01448408802
S315080024901549884203DC1248808888420ADD1148BB
S315080024A04038C07F002805D11049486005210D48ED
S315080024B04038C1770A4840880A2803DB08488088DC
S315080024C00A280ADA07484038C07F002805D1074994
S315080024D04860042103484038C1777FBDE8040020DE
S315080024E0740100202C040020E60F00000C020020D6
S315080024F000B587B001A800F0AFF80121480201F045
S315080025009DF900200190702002900120800203901E
S3150800251000200690059001A9064800F031F801212F
S31508002520044800F021F80121024800F011F807B02C
S3150800253000BD00000024014010B504460723002210
S315080025402146024800F038F810BD0000002401407A
S31508002550002904D0426801231A43426003E0426816
S315080025605208520042607047002904D08268082346
S315080025701A43826003E0826808239A4382607047A0
S3150800258042680B4B1A4042600B684A681A43436814
S315080025901A4342608268074B1A4082600B694A698F
S315080025A01A438B681A4383681A438260704700008F
S315080025B00FBCFFFF8FF1F9FFF0B504460D4616462E
S315080025C01F463F073F0F2B46082B0FD91B071B0F2C
S315080025D0083B606F9A000F21914088436067606FDF
S315080025E099003A468A40104360670BE0206F9A00CC
S315080025F00F21914088432067206F99003A468A4008
S3150800260010432067E0680121A9408843E060E0683C
S315080026100121A9400843E0600120800328400028E2
S3150800262003D0012000F020F807E00120C00328406D
S31508002630002802D0012000F017F8F0BD002905D0C7
S315080026408268FF2301331A43826004E08268FF230D
S3150800265001339A43826070470021016041608160BE
S315080026600173016141617047002806D0064949682F
S315080026700C221143044A516005E0034949680C22BB
S315080026809143014A516070470024014010B524481F
S315080026900078012834D10020214908702149088092
S315080026A012E02048008840001F49085A1F49098837
S315080026B0C9001F4A89181B4A1288520088521948AD
S315080026C00088401C17490880164800880428E8DB5B
S315080026D07E2002F07DFA022000F02EF9012115482D
S315080026E0FFF7ACFF11480088401C104908800846CF
S315080026F00088142804DB0020088001200E49087091
S315080027000D480078002806D0FFF78AFE00200A49FF
S31508002710087000F059FC7E2002F05AFA10BD00003D
S31508002720840100209E010020B0040020A0010020A2
S31508002730E8040020002401407C010020FFB583B096
S315080027400C46029400200190002726E000261CE093
S31508002750721C039951430846791CFFF7DBF80546B6
S31508002760A54201D9281B00E0601B05460298A8422D
S3150800277004D90295059806700698077002980028ED
S3150800278002D10120019002E0761C402EE0D300BF62
S315080027900198002800D002E07F1C042FD6D300BF82
S315080027A0029807B0F0BD000000BF00BF00BF00BF21
S315080027B000BFBFF34F8F00BF00BF00BF06480749E1
S315080027C0C86000BF00BF00BFBFF34F8F00BF00BF88
S315080027D000BF00BF00BFFDE70400FA0500ED00E0FA
S315080027E010B500F001F810BD10B523480078002890
S315080027F017D1224801F0AAF801283CD11F480078D1
S31508002800002838DD1D480078402834DC01F0BCFE7D
S315080028101B490860012018490870002019490870EA
S3150800282029E0164A17490978491C501801F08EF80C
S31508002830012816D113480078401C124908700F4821
S3150800284000780978884216D100200B4908700B4891
S315080028504078FF280FD10B48007802280BD1FFF7E4
S31508002860A3FF01F091FE064909686431884202D93E
S3150800287000200149087010BD490100206C040020A1
S315080028804C0100204801002010B586B004460121FD
S31508002890880300F0D3FF0121480400F0AFFF0122AE
S315080028A00921C80600F031FB01220A210920C006C9
S315080028B000F02BFB01A801F068FF0194302168465F
S315080028C0018100214181818101821821C18101A9EB
S315080028D0184801F017FF0121164801F0F0FE05A877
S315080028E000F069FB01214902684681820121817550
S315080028F01821C17505A90920C00600F0B9FA0121F9
S315080029008902684681824821C17505A90920C00641
S3150800291000F0AEFA1B2168460170032141700121BF
S31508002920817000F037FF01220221024801F0DFFE24
S3150800293006B010BD0038014001B506490098086088
S3150800294002E07E2002F044F9024800680028F8D127
S3150800295008BD000054010020014600220E4B1A61F2
S31508002960CA005A6100229A6105221A6100BF0A4A02
S315080029701069C207D20F002A04D0012212040240AD
S31508002980002AF4D0044A126952085200024B1A610E
S3150800299000229A617047000000E000E010B50021AF
S315080029A00448FFF74BFE022000F04AF801200249CE
S315080029B0087010BD002401408401002000B589B0CC
S315080029C00121084600F01AFF1A4800F045F801A848
S315080029D000F08EF8184801901848029000216846C1
S315080029E001730420049068460175802141754900E9
S315080029F0C182890001832021817609028183002111
S31508002A00C183018401A90B4800F04CF8012109484B
S31508002A1000F01CF801220221064800F039F80921C5
S31508002A2068460170022141700121817000F0B2FEF2
S31508002A3009B000BD0800024000240140B00400208F
S31508002A4001494860704700000000024002685208C9
S31508002A5052000A430260704710B5044620684008D1
S31508002A6040002060002020606060A060E060E1B265
S31508002A70084608380521FEF74DFF01460F20884015
S31508002A800249496808430149486010BD00000240F0
S31508002A90002A03D003680B43036002E003688B43F4
S31508002AA00360704710B50A7A8B7D1A430B7C1A436C
S31508002AB04B7C1A434B8A1A438B8A1A430B8B1A434D
S31508002AC04B8B1A430368094C23401A430260026879
S31508002AD00123DB039A438B8B1A430260CA68426060
S31508002AE00A6882604A68C26010BD00000F80FFFF56
S31508002AF00021016041600172C16001744174418224
S31508002B0081828175018341838183704770B506464A
S31508002B100C4621460A4800F04BF90546002D01D11E
S31508002B20401E70BD0648854202D10648051B00E0D6
S31508002B302D1B224629463046FEF716FF2046F0E7AB
S31508002B4000F4000800FC000870B506460C4621464D
S31508002B500A4800F02DF90546002D01D1401E70BD2A
S31508002B600648854202D10648051B00E02D1B224671
S31508002B7029463046FEF7F8FE2046F0E700A0000892
S31508002B8000A8000870B506460C4621460A4800F01B
S31508002B900FF90546002D01D1401E70BD0648854235
S31508002BA002D10648051B00E02D1B22462946304661
S31508002BB0FEF7DAFE2046F0E700B0000800B8000885
S31508002BC070B505460C4622460249284600F0B1F87B
S31508002BD0204670BD00F4000870B505460C4622462E
S31508002BE00249284600F0A5F8204670BD00A0000856
S31508002BF010B50446084800690221084306490861D9
S31508002C0008464461006940210843034908610348AE
S31508002C1000F00EF910BD000000200240FF0F000072
S31508002C200C48C068C007C00F002801D001207047B3
S31508002C300848C06804210840002801D00220F6E7A9
S31508002C400448C06810210840002801D00320EEE798
S31508002C500420ECE70020024003480069802108436D
S31508002C6001490861704700000020024030B504465B
S31508002C700D46054800690121084303490861258076
S31508002C800F2000F0D5F830BD0020024010B57E2098
S31508002C9001F09EFF064800F00FF87E2001F098FF2D
S31508002CA0044800F009F87E2001F092FF10BD0000EC
S31508002CB000F4000800A0000810B5044600F0ACF8BF
S31508002CC02046FFF795FFFFF7C7FF10BD70B503460F
S31508002CD00125002208E050001C5A0748844201D00A
S31508002CE0002506E0501C82B2CE0F76187610964262
S31508002CF0F1DC00BF284670BDFFFF0000F8B50546A9
S31508002D000E46144600F088F87E2001F061FF002781
S31508002D1007E029883046FFF7A9FFB61CAD1C781CCA
S31508002D2087B2E10F09194910B942F2DCFFF794FF9F
S31508002D30F8BDF8B507460C4615462946204600F064
S31508002D4037F80646002E0DD12046FFF7B5FF0120BD
S31508002D5080022018FFF7B0FF2A4621463846FFF7BB
S31508002D60CDFF24E0012080022018401BB0420AD182
S31508002D70012080022018FFF79FFF2A463146384671
S31508002D80FFF7BCFF13E00120C0022018401BB04229
S31508002D9008D12046FFF790FF2A4631463846FFF706
S31508002DA0ADFF04E02A4631463846FFF7A7FFF8BDCF
S31508002DB0F8B505460E462F46E807C00F002801D08D
S31508002DC000BFFEE731460120C002FEF7B9FD002923
S31508002DD001D000BFFEE700240BE0204670434719E8
S31508002DE031463846FFF772FF012800D108E0601C1B
S31508002DF084B231460120C002FEF7A2FDA042ECDCF7
S31508002E0000BF31460120C002FEF79AFDA04200D15C
S31508002E1000273846F8BD00000248034948600348C1
S31508002E20486070472301674500200240AB89EFCD13
S31508002E3010B5024600BFFFF7F3FE0346521EFF24F5
S31508002E4000E0641E002CFCD1012B01D1002AF2D12E
S31508002E500648006977218843044908613420C86018
S31508002E60002A01D1052010BD1846FCE700200240C3
S31508002E70F8B50246CD782F073F0FCD781026354096
S31508002E80002D01D08D782F431446002011E08506C9
S31508002E902B0E0D88012686403540002D07D0256863
S31508002EA00F269E40B5433E469E4035432560451C49
S31508002EB0E8B20828EBDB141D0D882D1200950020BA
S31508002EC011E085062B0E01258540009E3540002D14
S31508002ED007D025680F269E40B5433E469E4035439B
S31508002EE02560451CE8B20828EBDBCD78282D04D1EF
S31508002EF055690E883543556106E0CD78482D03D1CE
S31508002F0015690E8835431561F8BD70B54D07EB0E8A
S31508002F10082902DA0546203501E0054624352C46FF
S31508002F200F269E402568B54316469E4035432560C4
S31508002F3070BD000038B504460D460920C006844217
S31508002F4003D10121480400F059FC1148844203D1F9
S31508002F500121000200F052FC0E48844203D10121EF
S31508002F60000200F04BFC0C48844203D101210805FD
S31508002F7000F044FC684600F01EF86846058001210A
S31508002F8081700021C17069462046FFF771FF38BD80
S31508002F900004004800080048000C004802469068F3
S31508002FA00840002801D0012070470020FCE7416155
S31508002FB07047016170470021C94301800221817071
S31508002FC00421C1707047000000B591B000200F9031
S31508002FD00E900D900C907E2001F0FAFD00201090C6
S31508002FE01FE010984000FE49085A0590FEF751FF69
S31508002FF0FC490690FEF772FD0790FEF7BFFF002218
S31508003000F94B09910890FEF759FE0B910A90FEF7C5
S31508003010DDFF10998900F54A50501098401C80B27F
S31508003020109010980428DCDBF0488068F049069078
S31508003030FEF754FD0790FEF7A1FFEE4AEE4B099105
S315080030400890FEF733FE0B910A90FEF7BFFF0F902C
S31508003050E6484068E6490690FEF740FD0790FEF709
S315080030608DFFE44AE44B09910890FEF71FFE0B9189
S315080030700A90FEF7ABFF0E900F98FEF77FFF00222F
S31508003080D94B05910490FEF711FE09910890DB488B
S315080030900F99FEF7E6FC0590FEF770FF079106907C
S315080030A0099B089AFEF772FE0B910A90FEF78EFFAF
S315080030B0D34908600E98FEF761FF0022CA4B0591B6
S315080030C00490FEF7F3FD09910890CC480E99FEF797
S315080030D0C8FC0590FEF752FF07910690099B089ACF
S315080030E0FEF754FE0B910A90FEF770FFC54908607B
S315080030F0C548008D322830DAC448408B0190FEF767
S31508003100E3FEC34AC34B03910290FEF7D7FD0022A4
S31508003110C14B05910490FEF739FE09910890BB480A
S31508003120408B0290FEF7B5FEBC490390FEF7D6FC2D
S315080031300490B34801680498FEF78FFC0590FEF7E3
S315080031401DFF07910690099B089AFEF71FFE0B9133
S315080031500A90FEF73BFF0D905CE0AB48008DBE2859
S315080031602CDAAA48408B0690FEF793FE0890A748EB
S31508003170808B0590FEF78DFEA9490690FEF7AEFCFA
S3150800318007900899FEF76DFCA4490990FEF7A6FC7E
S315080031900B909E48408B0790FEF77BFE9F49089050
S315080031A0FEF79CFC0990964801680998FEF755FCBD
S315080031B00A900B99FEF792FC0D902BE09348408BF2
S315080031C00690FEF766FE08909048008C0590FEF77C
S315080031D060FE93490690FEF781FC07900899FEF772
S315080031E040FC8E490990FEF779FC0B908748408B86
S315080031F00790FEF74EFE89490890FEF76FFC099086
S315080032007F4801680998FEF728FC0A900B99FEF793
S3150800321065FC0D907C48408D322830DA7B48008B5F
S315080032200190FEF751FE7A4A7A4B03910290FEF717
S3150800323045FD0022784B05910490FEF7A7FD0991FC
S3150800324008907248008B0290FEF723FE734903909C
S31508003250FEF744FC04906B4801680498FEF7FDFBF2
S315080032600590FEF78BFE07910690099B089AFEF7D4
S315080032708DFD0B910A90FEF7A9FE0C905CE0624862
S31508003280408DBE282CDA6148008B0690FEF701FEB9
S3150800329008905E48C08B0590FEF7FBFD60490690D6
S315080032A0FEF71CFC07900899FEF7DBFB5B490990C3
S315080032B0FEF714FC0B905548008B0790FEF7E9FDC6
S315080032C056490890FEF70AFC09904E480168099885
S315080032D0FEF7C3FB0A900B99FEF700FC0C902BE057
S315080032E04A48008B0690FEF7D4FD08904748408C64
S315080032F00590FEF7CEFD4A490690FEF7EFFB0790CC
S315080033000899FEF7AEFB45490990FEF7E7FB0B90D7
S315080033103E48008B0790FEF7BCFD40490890FEF733
S31508003320DDFB0990374801680998FEF796FB0A9075
S315080033300B99FEF7D3FB0C903A480D99FEF738FB2C
S315080033400B90FEF7E8FD3849086036480C99FEF7F9
S315080033502FFB0B90FEF7DFFD344908602A48008DE5
S31508003360314909684018C003010C27480185408D7A
S315080033702E4909684018C003010C234841851B489B
S31508003380C0682B490A90FEF76CFB0B90FEF7C3FD4D
S3150800339081B21D480187FF38C1380088FF21F53101
S315080033A0884276DD00201949683908800F48006888
S315080033B00990FEF7E3FD1F4A1F4B0B910A90FEF793
S315080033C0F1FD56D2094800680990FEF7D7FD1B4A59
S315080033D01B4B0B910A90FEF7E5FD45D2402131E0E3
S315080033E07401002000F07F4500000840D804002042
S315080033F00000404125068195438BD43F0000484391
S315080034008C01002090010020CC03002074020020CB
S31508003410091B9E5E29CB703F00408F4000007A440E
S31508003420002474490000C841940100209801002036
S315080034300000C842736891ED7C3FDD3F9CC420B014
S315080034407268D13F2B48FFF7A9FD00280CD12A48FE
S31508003450407F012808D12848C07F002804D1274981
S31508003460486006212448C177012023494031087164
S3150800347014E02348006823490B90FEF7CDFD0DD2D2
S315080034801D484030407B002804D11B494031087153
S3150800349004E02CE0012018494031087118480068FA
S315080034A019490B90FEF7B8FD04D2012112484030A5
S315080034B0417103E000211048403041710E48403008
S315080034C0007900280ED10C48407F012804D101025A
S315080034D00848FFF76CFD0AE0FF2101310548FFF7B0
S315080034E068FD04E0FF2101310248FFF762FD11B0D3
S315080034F000BD000000040048EC0300200C02002078
S31508003500D80400206F12233F333313400148806AE2
S3150800351070470000C0F7FF1F0148006870470000A9
S3150800352058010020034800680349097840180149F2
S3150800353008607047580100206001002008B5012185
S31508003540480400F05BF90121880400F057F9684641
S31508003550FFF731FD0121C903684601804821C17082
S3150800356069460920C006FFF783FC6846FFF723FD76
S3150800357001210903684601804821C170694609206E
S31508003580C006FFF775FC6846FFF715FD402168463B
S3150800359001800421C17069460148FFF769FC08BD2E
S315080035A00004004810B50121C9030920C006FFF729
S315080035B0F5FC002841D154488078002831D152487A
S315080035C02038407F012829D14F482030407B0028E9
S315080035D024D14E480078401C4C49087008460078AB
S315080035E005281BDB0020087004214948FFF7E1FC89
S315080035F0454898384089002807D1464846494860D2
S31508003600012141489838418106E000204249486036
S3150800361000213D489838418101F0FAFA01213A48DB
S3150800362081703E480078002810D101203B49087077
S31508003630012135482038817708E00020374908708D
S315080036400021314820388177203081703248C0689F
S315080036503049884251D900202F49C86000212A489C
S31508003660203881774030407B00283FD10821284800
S31508003670FFF79FFC24489838408803283DDA2248FB
S3150800368098384089002838D11F484038408D82280C
S3150800369010DA1D482030407900280BD11A48203806
S315080036A0407F012829D118492031487300201A493A
S315080036B0486022E014482038407F012802D10020C3
S315080036C01549486010484038408D822804DB02219D
S315080036D00D482038C17710E00B4820304079012882
S315080036E00BD1012108482038C17706E000200A4995
S315080036F0486000210448203841777E2001F068FAA6
S3150800370001482038807F10BD0C040020C40000202A
S3150800371000040048DC0500000C020020A20100207D
S3150800372008B50121480400F069F80121880400F071
S3150800373065F86846FFF73FFCFF210E3168460180B1
S31508003740012181701021C17069461148FFF790FB6D
S31508003750B62168460180012181701021C170694631
S315080037600920C006FFF784FB10210920C006FFF7D1
S315080037701EFC80210920C006FFF719FC0121044818
S31508003780FFF715FC08210248FFF713FC08BD0000E7
S31508003790000400488178002925D01749032212021F
S315080037A08918027892109200895802789207D30EE7
S315080037B0FF229A40914342789207120E03789B079C
S315080037C0DB0E9A4011430C4A03231B02D2180378D6
S315080037D09B109B00D1500178CA06D20E0121914058
S315080037E0054A116007E00178CA06D20E0121914008
S315080037F0014A80321160704700E100E0002905D0D7
S31508003800054A52690243044B5A6104E0024A526966
S315080038108243014B5A61704700100240002905D0C7
S31508003820054AD2690243044BDA6104E0024AD269C6
S315080038308243014BDA61704700100240002905D027
S31508003840054A92690243044B9A6104E0024A926966
S315080038508243014B9A6170470010024010B500F090
S3150800386031F804494968F02211400909024A515CB5
S31508003870C84010BD001002402201002010B5FFF715
S31508003880EDFF05494968072212021140090A034A51
S31508003890515CC84010BD0000001002402201002003
S315080038A010B5FFF7DBFF054949680722D202114028
S315080038B0C90A034A515CC84010BD00000010024006
S315080038C022010020F8B51E4840680C21084004284B
S315080038D002D008282ED101E01A4C2DE018484030B5
S315080038E00069C007C00F00280AD015484030006993
S315080038F002210840002801D0134802E0114800E0E0
S31508003900104807460E4840300069FF210904084060
S31508003910000C451C0A484030006907210902084086
S31508003920000A461C3946694308463146FDF7F2FF48
S31508003930044601E0034C00BF00BF2046F8BD000066
S315080039400010024000127A0000093D0070B50446D6
S3150800395000250221074800F0B8FE002808D00548CF
S3150800396000F00CFF20700221024800F0A6FE012597
S31508003970284670BD0038014010B500F001F810BDAA
S3150800398000B585B0624800680121084360490860AF
S3150800399000BF5F480068022108400028F9D05D484A
S315080039A05D4908605D480068102108435B49086066
S315080039B008460068C008C000086057490968481EDC
S315080039C05749FDF7A7FF049054480068049949072A
S315080039D0490F0843514908604D4840685149084015
S315080039E04B49486008464068902108434849486062
S315080039F0084640684860484800684649884207D9EA
S31508003A0043484068052109020843414948600BE0DC
S31508003A10414800684449884206D93D484068012122
S31508003A20890208433A4948606B4601AA3A48016840
S31508003A303E48FEF783FE364840300069800880001D
S31508003A40334940310861084600694008400008616A
S31508003A50684600784007400F02906846007940069D
S31508003A60400E03902A48C069890508432849C86159
S31508003A702748403000692E490840254940310861E9
S31508003A80039800040299090208432149403109694B
S31508003A9008431F49403108611D480068012109068D
S31508003AA008431B49086000E000BF19480068012167
S31508003AB0490608400028F7D0154840688008800065
S31508003AC0134948600846406802210843104948607F
S31508003AD000E000BF0E4840680C2108400828F8D1CD
S31508003AE00120FEF739FF0A48406810218843084933
S31508003AF048600120FEF730FF05484068802188436A
S31508003B00034948600120FEF727FF05B000BD000005
S31508003B100010024000A24A0434010020002002409E
S31508003B2000366E010FC0FFFF0051250200127A0011
S31508003B30FFF800FF042806D1064909690422114343
S31508003B40044A116105E00349096904229143014ABF
S31508003B501161704700E000E010B5FFF7E3FC9148FB
S31508003B600088401C8F49088008464068401C486009
S31508003B708D480088401C8C4908808C4800680028BD
S31508003B8004D08A480068401E884908608848807FB3
S31508003B90012805D18348C068401C8249C86002E0F4
S31508003BA000208049C86082484030807A012805D1C3
S31508003BB07C484069401C7B49486102E000207949FD
S31508003BC048617B4820300078012805D17548006C8B
S31508003BD0401C7449086402E000207249086471496F
S31508003BE048680A21FDF796FE002923D1704820303F
S31508003BF0C17F807F814208DD6D482030807F401C70
S31508003C00C1B26B482030817714E069482030C17F03
S31508003C10807F814200D10DE065482030C17F807FDA
S31508003C20814207DA62482030807F401EC1B2604870
S31508003C30203081775E484030407B022804D05C48BB
S31508003C404030407B032804D15648806B401C5549B8
S31508003C50886357484030407800280AD15448403095
S31508003C60407B042805D14F48806C401C4D49886428
S31508003C7002E000204B4988644D484030407B0028CC
S31508003C8003D148490865C86428E049482030C07807
S31508003C90012805D14348006D401C4249086502E0E9
S31508003CA0002040490865424820300079012812D191
S31508003CB03C48C06C401C3B49C8643D48403080784D
S31508003CC0002804D108468068401C886006E0002069
S31508003CD03449886002E000203249C8643448807E4E
S31508003CE004280AD12F48406D3249884208D22D4807
S31508003CF0406D401C2B49486502E00020294948656B
S31508003D00012109030920C006FFF748F9002813D046
S31508003D1027484030007900280ED12548407F0128E1
S31508003D200AD12048806D2449884208D21D48806DF2
S31508003D30401C1C49886502E000201A4988651C4811
S31508003D404030807901280AD11648C06D1B4988423F
S31508003D5008D21448C06D401C1249C86502E000200C
S31508003D601049C86512484030007A012805D10D4827
S31508003D70006E401C0B49086602E0002009490866E7
S31508003D800B484030407A012805D10648406E401C51
S31508003D900449486602E00020024948667E2000F091
S31508003DA017FF10BD0C02002050010020540100200E
S31508003DB0EC03002050C300008813000070170000B1
S31508003DC010B51648006801210843144908600846DA
S31508003DD04068134908401149486008460068114977
S31508003DE008400E490860084600680121890488438E
S31508003DF00A49086008464068C321090488430749F8
S31508003E0048600846006808490840044908609F2039
S31508003E1000048860FFF7B0FD10BD000000100240E6
S31508003E200CC0FFF8FFFFF6FEFFFF8F0008B5012163
S31508003E304804FFF7E3FC022201210920C006FFF728
S31508003E4064F80221684601801821C1700121817039
S31508003E5069460920C006FFF70BF801214804FFF759
S31508003E60CDFC022211460920C006FFF74EF80421B0
S31508003E70684601801821C1700121817069460920B0
S31508003E80C006FEF7F5FF08BD30B587B004460D46F7
S31508003E9001210846FFF7C2FC04A800F033F905948F
S31508003EA068460582002101838176817404A9012070
S31508003EB0800700F0F1F8684600F0D2F860216846FD
S31508003EC001700121417000200190002168460172AD
S31508003ED069460120800700F057F8694601208007E7
S31508003EE000F08AF80821C80600F07EF80821C806FE
S31508003EF000F0B0F84021080600F038F8402108061E
S31508003F0000F03CF80121880700F00AF8012188072B
S31508003F1000F01EF80121880700F00EF807B030BD42
S31508003F20002904D0026880231A43026003E002686D
S31508003F3080239A4302607047002904D0026801234F
S31508003F401A43026003E00268520852000260704792
S31508003F50002905D0426C0123DB031A43426404E0BE
S31508003F60426C0123DB039A43426470478269072344
S31508003F701B039A430B021A4382617047C269702376
S31508003F809A430A43C261704710B5826907231B0327
S31508003F909A430B781B021A4382610A7A12014B78FC
S31508003FA01B011A43036A3024A3431A4302624A6870
S31508003FB082630C4A904213D14A7A12018B781B010C
S31508003FC01A43036AC024A3431A4302624A89920029
S31508003FD08B899B001A4343682401A3431A43426012
S31508003FE010BD0000002C014082690123DB029A43C0
S31508003FF00B021A438261704710B5C26970239A434F
S315080040000B781A43C2610A7A12024B781B021A43CA
S31508004010036A03242402A3431A4302624A68C2635A
S315080040200B4A904213D14A7A12028B781B021A4322
S31508004030036AA400A3431A4302624A8912018B89C0
S315080040401B011A434368A400A3431A43426010BDE8
S31508004050002C0140C26908239A430A43C26170478B
S315080040600021017041708170416001724172418185
S315080040708181704701229207904201D1816301E054
S315080040808AB28263704701229207904201D1C163C6
S3150800409001E08AB2C2637047026803231B029A438F
S315080040A00B891A430260134A904206D001229207EE
S315080040B0904202D0104A904205D1026870239A4372
S315080040C08B781A4302600B4A904205D00B4A9042FD
S315080040D002D00B4A904205D1026B120A12028B7A61
S315080040E01A4302634A68C2620A88826201224261EE
S315080040F070470000002C01400004004000440140C5
S31508004100004801400021C943416000210180018126
S31508004110817081727047000010B50024FA48807AD1
S3150800412000280FD1F9484068F9490968401AF94941
S3150800413088420BD90021F448403841770020F249DB
S31508004140487303E0F1484068F1490860EE48C079D1
S31508004150030000F0B4FD050478F1EFEEED00EA493E
S3150800416020398A8BE9494868B32104F05FFC044684
S31508004170E5482038408B912805DA0F2201210020D6
S3150800418002F000F804E000220121104601F0FAFFCF
S31508004190DD482038808BB42809D0DB482038808B4E
S315080041A0B32804D0D8482038808BB52813D1D648F0
S315080041B06038408DD8490988884208D00020D249FD
S315080041C0487208466038408DD349088006E00120C9
S315080041D0CD49487202E00020CB494872CB48406E70
S315080041E0CE49884226D9C8482038408B801ECC49FB
S315080041F00988884216DCC4482038408B801CC84988
S31508004200098888420EDBC6480088A5280FDB02F01D
S3150800421039FC0120BC49C8710020BC494866C1491F
S31508004220087004E0B8482038408BBD490880002053
S31508004230B64948660020BC4908702246012108464E
S3150800424001F0A0FF97E1B04920390A8BAF494868C9
S31508004250B32104F0EBFB044600220121084601F0D5
S3150800426091FFA9482038008BB42809D0A6482038E1
S31508004270008BB32804D0A4482038008BB52813D166
S31508004280A1486038008DA4490988884208D00020D2
S315080042909D49487208466038008D9F49088006E0A7
S315080042A001209949487202E00020974948729748C8
S315080042B0406E9A49884222D993482038408B801EFE
S315080042C097490988884212DC8F482038408B801C21
S315080042D09349098888420ADB02F06CFC02208A4965
S315080042E0C8710020894948668E49087004E08648E6
S315080042F02038408B8A4908800020844948668A48C5
S31508004300007800280ED180482038808B822805DD69
S3150800431000220121104601F035FF08E001208249FC
S31508004320087004E022460121002001F02BFF22E15B
S3150800433020E107E16BE0FFE7734920398A8B73496F
S315080043404868E52104F072FB044600220121104664
S3150800435001F018FF6C482038808BE62809D06A4897
S315080043602038808BE52804D067482038808BE728DA
S3150800437013D165486038408D67490988884208D056
S3150800438000206149487208466038408D62490880B5
S3150800439006E001215C48417202E000215A48417258
S315080043A05A48406E5D49884228D957482038408B7C
S315080043B0801E5B490988884218DC53482038408BA0
S315080043C0801C57490988884210DB55480088D2283E
S315080043D011DB02F087FC03204B49C87102F01EFB73
S315080043E000204A4948664F49087004E04648203884
S315080043F0408B4B49088000204449486600204B49B9
S31508004400087022460121084601F0BCFEB3E03E4989
S3150800441020390A8B3D494868E52104F007FB044624
S3150800442000220121084601F0ADFE37482038008BEE
S31508004430E6280BD034482038008BFF212C318842DF
S3150800444004D031482038008BE72813D12E4860382D
S31508004450008D31490988884208D000202A494872C7
S3150800446008466038008D2C49088006E00120264958
S31508004470487202E00020244948722448406E2749C1
S31508004480884231D920482038408B801E2449098823
S31508004490884221DC1C482038408B801C204909882A
S315080044A0884219DB1E480088C3281ADB1C48008886
S315080044B0D22816DA02F0AEFC04201349C87102F0BD
S315080044C0ADFA0122FE21572003F0C1FA00200F4958
S315080044D048661449087004E00B482038408B104998
S315080044E0088000200949486610480078002823D12A
S315080044F005482038408BC8281ADD002201211046BD
S3150800450001F040FE1DE000002C0400200C020020F3
S3150800451010010020C409000016010020DC05000077
S315080045200C010020F80000201801002019010020C5
S3150800453001201249087004E022460121002001F0FA
S3150800454021FE18E00E494868FF21F531FDF7E2F92A
S3150800455000290ED100200A4948660A4948850022E2
S315080045600121104601F00EFE00220121084601F045
S3150800457009FE00E000BF00BF10BD000019010020C1
S315080045800C0200203C04002010B5FEF7C5FF10BD44
S3150800459070B5FFF763F905467D21C900FDF7BAF93D
S315080045A00446601E0C49884200D90CE0601E0B497F
S315080045B048610321081F00F091FB00200749886124
S315080045C00720086100BF0420FFF7B4FA0021481E3F
S315080045D000F084FB70BD0000FFFFFF0000E000E074
S315080045E010B50221134800F079F8002820D01148A8
S315080045F000F0C4F8C4B21048C07E022811D10E4893
S31508004600007F002810D10D488079AA2804D10B48CC
S31508004610C471012108480177AA2C05D1074884717D
S3150800462002E0204602F08EFC0221024800F045F81E
S3150800463010BD000000380140EC030020980500205A
S3150800464010B504462146054800F09CF800BF012134
S31508004650024800F03AF80028F9D010BD00380140A9
S3150800466070B505460E4600247E2000F0B1FA00BF5C
S3150800467020E0042C19DD701EA04216DD285D7E2878
S3150800468006D17D20FFF7DCFF5E20FFF7D9FF0FE09C
S31508004690285D7D2805D1FFF7D3FF5D20FFF7D0FF02
S315080046A006E0285DFFF7CCFF02E0285DFFF7C8FFAC
S315080046B0601C84B2B442DCDB70BD4161704782691C
S315080046C0520852000A4382617047024690680840C1
S315080046D0002801D0012070470020FCE70246D06878
S315080046E00840002801D0012070470020FCE7002A76
S315080046F003D003690B43036102E003698B4303613B
S315080047007047000070B504460D460026E069302162
S31508004710884329790843E061E06944218843A979F7
S315080047200843E061E06980088000297A0843E0616F
S31508004730A0691821884369890843A061A0690421F2
S315080047408843297B0843A0610B48844203D1FFF7BD
S31508004750A7F8064602E0FFF791F8064630462968AC
S31508004760FDF7D8F80009206230462968FDF7D2F827
S315080047700007000F606270BD0038014001464868B6
S31508004780C0B27047CAB2026070474B21C9010160C6
S3150800479030210171002181710172182141810021A6
S315080047A00173704710B51C484088030000F087FA6B
S315080047B00504111E292A2B0017485830008FFF219F
S315080047C01B31884204DA01211348418000F020FA9F
S315080047D019E011485830008FFF210531884204DA64
S315080047E002210D48418000F013FA0CE00A485830BF
S315080047F0008FF62804DA03210748418000F008FAFA
S3150800480001E000E000BF00BF03487830407F002881
S3150800481001D100F0FDF910BD7403002010B5304831
S315080048204088002806D0012813D0022820D0032863
S3150800483054D12CE080210920C006FEF7BAFB0121DD
S315080048402848FEF7B6FB10210920C006FEF7B1FB83
S3150800485044E001212348FEF7ACFB80210920C0066D
S31508004860FEF7A5FB10210920C006FEF7A0FB35E0E0
S3150800487080210920C006FEF79CFB01211948FEF796
S3150800488096FB10210920C006FEF791FB26E0164983
S315080048904868CD21FDF73EF8C007C00F002805D1AE
S315080048A080210920C006FEF782FB0DE00E49486804
S315080048B0CD21FDF72FF8C007C00F002804D08021AE
S315080048C00920C006FEF775FB01210648FEF76FFBB7
S315080048D010210920C006FEF76AFB00BF00BF10BD05
S315080048E074030020000400480C02002010B59F48FD
S315080048F0807E030000F0E3F90504336CAFFAF80094
S315080049009A482038008FFF211031884202DB0121A6
S315080049109648817640219648FEF740FB00281DD030
S3150800492094494868FF21F531FCF7F4FFC007C00F2A
S31508004930002805D180210920C006FEF738FB04E0CF
S3150800494080210920C006FEF734FB10210920C00685
S31508004950FEF72DFB01218648FEF729FB03E1834874
S315080049602038008FFF212531884202DB02217F484B
S31508004970817640217E48FEF711FB002827D07D4925
S315080049804868FF21F531FCF7C5FFC007C00F0028AE
S3150800499004D101217648FEF70AFB03E00121744899
S315080049A0FEF707FB80210920C006FEF700FB102151
S315080049B00920C006FEF7FBFA6C48783840880128BB
S315080049C005D0012169487838418000F021F9CAE00C
S315080049D066482038008FFF212731884202DD0321EF
S315080049E06248817640216248FEF7D8FA002831D01D
S315080049F060494868FF21F531FCF78CFFC007C00FF6
S31508004A0000280ED180210920C006FEF7D2FA01211E
S31508004A105748FEF7CEFA10210920C006FEF7C9FA54
S31508004A200DE080210920C006FEF7C1FA10210920F1
S31508004A30C006FEF7BCFA01214D48FEF7B8FA4B4806
S31508004A4078384088002805D00021484878384180C1
S31508004A5000F0DEF887E040214548FEF79FFA002877
S31508004A6041D0012109030920C006FEF797FA00285C
S31508004A7007D04048806D4049884202D904213B4806
S31508004A8081763C494868FF21F531FCF743FFC007AA
S31508004A90C00F00280ED180210920C006FEF789FA2A
S31508004AA001213348FEF785FA10210920C006FEF7D2
S31508004AB080FA0DE080210920C006FEF778FA102159
S31508004AC00920C006FEF773FA01212948FEF76FFA96
S31508004AD0264878384088002805D0002123487838A9
S31508004AE0418000F095F83EE03CE0FFE74021204891
S31508004AF0FEF754FA002834D01C4878384088002835
S31508004B0005D0002119487838418000F081F8194805
S31508004B10406D1A4988420ED280210920C006FEF748
S31508004B2048FA01211248FEF744FA10210920C00666
S31508004B30FEF73FFA0DE080210920C006FEF737FA96
S31508004B4010210920C006FEF732FA01210848FEF7AF
S31508004B502EFA064840300079012802D1032103487D
S31508004B60817600E000BF00BF10BD0000EC03002006
S31508004B70000400480C020020941100003075000063
S31508004B800348806840084000014988607047000073
S31508004B90002C004080210143014A11607047000043
S31508004BA0002C004003488068002801D00120704787
S31508004BB00020FCE7002C004010B5FFF7F3FF0028A3
S31508004BC004D0FFF7DDFF662000F002F810BD0000F4
S31508004BD04106490E014A116070470000002C00404A
S31508004BE004494968FF22813291430143014A5160D1
S31508004BF070470000002C004004494968C909C901EA
S31508004C004206520E1143014A51607047002C00407B
S31508004C1010B57E20FFF7DCFF0948FEF74DF8094975
S31508004C20094801850621283000F018FA0649283176
S31508004C3088814022024904482830FEF77AF810BDD8
S31508004C4000B00008FBAA00004C03002070B505461A
S31508004C500C460121C802FEF7E1FDFF208130FFF76F
S31508004C60BFFF2046FFF7C8FF2846FFF793FF70BD32
S31508004C700FB410B503A9044B044A029800F080F853
S31508004C8010BC08BC04B01847616A0008040200207A
S31508004C902021020C01D010211046020A01D010462C
S31508004CA00839020901D01046091F820801D01046AA
S31508004CB0891E420801D0881E7047081A704730B40A
S31508004CC07446641E2578641CAB4204D3635D5B009E
S31508004CD0E31830BC18471D46F8E7000010B5002851
S31508004CE019DB1A4A03231B02D21883089B00D258E1
S31508004CF08307DC0EFF23A3409A438B071B0E84070A
S31508004D00E40EA3401A43114B032424021B198408FA
S31508004D10A4001A5118E00E4A03071B0F083B9B080C
S31508004D209B00D2588307DC0EFF23A3409A438B07C8
S31508004D301B0E8407E40EA3401A43054B0407240FF1
S31508004D40083CA408A4001A5110BD000000E100E0C8
S31508004D501CED00E002E008C8121F08C1002AFAD1BB
S31508004D6070477047002001E001C1121F002AFBD1DD
S31508004D7070470000014908607047000008020020DB
S31508004D80FFB58FB00F460446002606E025280AD050
S31508004D90129A11999047641C761C20780028F5D140
S31508004DA0304613B0F0BD00250121A14A009500E068
S31508004DB00543641C23780846203B98401042F7D1E7
S31508004DC020782E2815D1042005436078641C2A28EB
S31508004DD00AD101CF641C00900BE000990A225143C6
S31508004DE030394018641C009020780146303909296A
S31508004DF0F3D920786C280ED004DC4C2813D06A2806
S31508004E0012D104E074280ED07A280DD10BE00120C7
S31508004E104005054307E00121090562780D438242F2
S31508004E2001D16D18641C641C2078864669284AD00E
S31508004E3008DC0028B4D058286DD0632810D0642820
S31508004E4008D140E070286BD0732812D0752860D03E
S31508004E50782860D0129A704611999047761CE5E03A
S31508004E603878694608720020487202A80190012025
S31508004E7003E0386801900020C0433F1D69070CD540
S31508004E80002500E06D1C00998D420FDA8542F9DB9A
S31508004E900199495D0029F5D108E0002500E06D1C5F
S31508004EA08542FCDB0199495D0029F8D1761907E0AE
S31508004EB0019801990078491C0191129A1199904715
S31508004EC06D1EF5D2B2E00A20029000216802400F5A
S31508004ED0039102280CD001CFC117844600290DDAA8
S31508004EE06246084652420021814194462D2008E038
S31508004EF0FF1DFF08FF0003CF8446EFE7280504D50A
S31508004F002B206A46107401203CE0E8073AD020209E
S31508004F10F7E70A2000E0102000210391029007E03D
S31508004F2010200290002104200543082003910090D8
S31508004F306802400F022810D001CF002184460020C5
S31508004F400D9028071FD5704670280CD0029A10209D
S31508004F50039B42401A430CD015E0FF1DFF08FF00D3
S31508004F6003CF8446EBE740206A46107401200D9073
S31508004F700CE06046084306D030206A461074704636
S31508004F80507402200D907046582804D029A001902C
S31508004F900DA80E900DE02CA0F9E76046039B029A37
S31508004FA0FDF744F8019B84469B5C0E9A521E0E92AE
S31508004FB0137060460843F0D10E9805A9081A2030E8
S31508004FC00190680701D5009801E001200090019939
S31508004FD0884203DD01460198081A00E000200025F2
S31508004FE0009006E004A8129A405D119990476D1C3E
S31508004FF0761C0D988542F5DB04E0129A302011994B
S315080050009047761C0099481E00900029F5DC08E0B8
S315080050100E980E990078491C0E91129A119990478C
S31508005020761C0199481E01900029F1DC641CB4E63F
S315080050300928010030313233343536373839616260
S315080050406364656600000000303132333435363724
S3150800505038394142434445460000000010B502462F
S315080050600023002901D1002010BD03E01488921CFA
S31508005070E01883B208464C1EA1B20028F6D118469D
S31508005080F2E7000010B5C148407F002865D110211D
S315080050900920C006FDF78BFF80210920C006FDF711
S315080050A086FF0121BA48FDF782FF0020B749403143
S315080050B04873002301221946184602F065FD0023AD
S315080050C01A461946184602F05FFDB2484068FF21A5
S315080050D0F531884204D20421AD48FDF76AFF53E151
S315080050E00421AB48FDF763FFAA484068AA498842ED
S315080050F0F5D9A64820308078002817D1A5484068F9
S315080051007D214901884201D2FFF74CFB0821A048BE
S31508005110FDF74DFF00219D48C17700209B4940318E
S31508005120487088709B49486248630CE0402198485B
S31508005130FDF734FF002806D000219448403041731B
S3150800514001214038417720210920C006FDF72FFFAD
S315080051507D2040018F49486016E18C484030407BED
S315080051600300FFF7ACFD060471B4FDFCFB700020DC
S3150800517086494031487088708649486248630023EA
S3150800518001221946184602F0FFFC00231A46194662
S31508005190184602F0F9FC7D482038418D01862030FA
S315080051A0C07E012808D17B4840697C49884202D9DB
S315080051B000217648C17610BD764840687D210901F0
S315080051C0884228D9002076490870704820308078AF
S315080051D0002802D16F49486002E072486D4948606C
S315080051E040216B48FDF7DAFE00280CD1FFF7DAFA02
S315080051F008216748FDF7DBFE7E20FFF7E9FC1E2045
S31508005200FDF79AFB02E000206249486004216048E5
S31508005210FDF7CDFE17E020210920C006FDF7C9FEDF
S3150800522008215B48FDF7C5FE5A484068FF21F5315D
S31508005230884208D9554878384089002803D104217E
S315080052405348FDF7B4FE9EE052484068FF21F53109
S31508005250884204D204214E48FDF7ABFE03E0042140
S315080052604B48FDF7A4FE4948C07E052817D1002201
S315080052700121084600F086FF44482038018D403059
S31508005280C08A814205DA64220121002000F07AFFF3
S3150800529007E000220121104600F074FF01E0FEF746
S315080052A03BFF3A482038418D4030C08A81420DDBA9
S315080052B036482038018D4030C08A814206DB0020FE
S315080052C03449486002203149403148735BE031482F
S315080052D04068FF21F531884204D204212C48FDF7A5
S315080052E068FE03E004212A48FDF761FE2948406864
S315080052F02D49884221D925482030C08AD2281CD178
S3150800530022482030808BCF2813DB20482030808B22
S31508005310D5280EDA01201D49403108721D48006E55
S315080053201E49884209D90122FE21672002F08FFB17
S3150800533003E000201549403108721448C07E05284C
S315080053401BD100220121084600F01CFF0F48203817
S31508005350018D4030C08A814209DA02E012E010E08D
S315080053600EE03C220121002000F00CFF07E000229D
S315080053700121104600F006FF01E0FEF7CDFE02E02F
S3150800538001E000E000BF00BF00BF14E7EC03002007
S31508005390000400480C020020B80B00008813000027
S315080053A0C4000020C40900001027000010B5C0483A
S315080053B0407F002865D110210920C006FDF7F7FDBA
S315080053C080210920C006FDF7F2FD0121B948FDF745
S315080053D0EEFD0020B64940314873002301221946E4
S315080053E0184602F0D1FB00231A461946184602F061
S315080053F0CBFBB1484068FF21F531884204D204212D
S31508005400AC48FDF7D6FD50E10421AA48FDF7CFFDCB
S31508005410A9484068A9498842F5D9A5482030807826
S31508005420002817D1A44840687D214901884201D245
S31508005430FFF7B8F908219F48FDF7B9FD00219C48F8
S31508005440C17700209A494031487088709A49486265
S3150800545048630CE040219748FDF7A0FD002806D0D8
S315080054600020934940314873012191484177202112
S315080054700920C006FDF79BFD7D2040018E49486046
S3150800548013E18B484030407B0300FFF718FC060405
S3150800549075B1FDFCFB740020854940314870002138
S315080054A0834840308170002083494862486300235E
S315080054B001221946184602F067FB00231A461946C8
S315080054C0184602F061FB7A482038418D0186203063
S315080054D0C07E012808D1784840697949884202D9AE
S315080054E000217348C17610BD734840687D210901C3
S315080054F0884228D90020734908706D482030807882
S31508005500002802D16C49486002E06F486A49486041
S3150800551040216848FDF742FD00280CD1FFF742F903
S3150800552008216448FDF743FD7E20FFF751FB1E2046
S31508005530FDF702FA02E000205F49486004215D4851
S31508005540FDF735FD17E020210920C006FDF731FDDE
S3150800555008215848FDF72DFD57484068FF21F531C9
S31508005560884208D9524878384089002803D104214E
S315080055705048FDF71CFD97E04F484068FF21F5317C
S31508005580884204D204214B48FDF713FD03E00421A9
S315080055904848FDF70CFD4648C07E062817D100226C
S315080055A00121104600F0EEFD41482038418D40307B
S315080055B0C08A814205DA50220121084600F0E2FD40
S315080055C007E000220121084600F0DCFD01E003F0B7
S315080055D07FF937482038418D4030C08A814206DB42
S315080055E000203549486002203149403148735BE064
S315080055F031484068FF21F531884204D204212D48FC
S31508005600FDF7D7FC03E004212A48FDF7D0FC2A4819
S3150800561040682E49884221D925482030C08AD22898
S315080056201CD123482030808BCF2813DB204820301C
S31508005630808BD5280EDA01201D49403108721E4894
S31508005640006E1F49884209D90122FE21672002F00F
S31508005650FEF903E000201649403108721448C07E5E
S3150800566006281BD100220121104600F08BFD1048A8
S315080056702038418D4030C08A814209DA3C22012116
S31508005680084602E00FE00DE00BE000F07BFD07E0C6
S3150800569000220121084600F075FD01E003F018F923
S315080056A002E001E000E000BF00BF00BF1BE700000A
S315080056B0EC030020000400480C020020B80B000090
S315080056C088130000C4000020C40900001027000049
S315080056D0F0B587B0002006900590002400250490B8
S315080056E000260027F948807A012815D1F84840692C
S315080056F07D21090188420FD90021F44881720020D2
S31508005700F3494861F3490880F3490870FF210131DC
S31508005710F048801DFCF741F9EC484038007F012825
S3150800572077D17E20FFF754FAEA48C0790002E949A2
S31508005730097A08430690E748407A0590E548847A4E
S31508005740C67A0246117B507B01F050FD0746E14AB6
S31508005750D17A107B01F04AFD05460021DB48403826
S3150800576001770121403081720020D9494861DB4A1E
S315080057700698811A90427AD02EDCD94A811A90422C
S3150800578076D016DCD74A811A904272D00ADC4428B1
S3150800579032D0D549401800286CD001286BD0022891
S315080057A06AD140E2012968D0022967D00329F7D1D6
S315080057B08EE2312970D008DC0D296ED00E296DD005
S315080057C00F296CD03029EBD167E3382968D04129F5
S315080057D067D05229E4D1C3E30B00FFF770FA174DDF
S315080057E0F1F0EFF2EDEC4D4D4D4DC1D9EBEA4D4DD3
S315080057F0222E88A250704D00059806280AD1BB486B
S31508005800007800280CD102F05FF90120B74908702A
S3150800581006E0B8E30598152802D1012002F054F9EC
S31508005820B0E3AA48407B002806D0A8486038028D15
S31508005830418D002002F068F8A4E3002C0AD1A348A1
S315080058406038408D00231A46F0210090FE2002F0B1
S31508005850CAF80BE0012C09D19C486038008D012359
S315080058600022F0210090FE2002F0BDF88AE36CE1E8
S3150800587054E2F0E1B4E1C2E183E30AE214E2002C67
S3150800588010D193486830408800231A46F3210090C7
S31508005890FE2002F0A8F811E000E362E2ACE2F6E2CC
S315080058A0FDE22BE3012C09D1894868308089012360
S315080058B00022F3210090FE2002F095F862E3002C06
S315080058C003D183486830458002E081486830858185
S315080058D07F4868308089FF21F531884206DA01F071
S315080058E09DF80022FE21F42002F0B1F84AE3002CCC
S315080058F00AD177486830808800231A46F12100903B
S31508005900FE2002F070F80BE0012C09D170486830CF
S31508005910C08901230022F1210090FE2002F063F8DD
S3150800592030E3002C03D16A486830858004E0012CF6
S3150800593002D167486830C581654868308088FF218C
S31508005940F53188420BDC62486830C089884206DC3B
S3150800595001F064F80022FE21F22002F078F811E343
S31508005960002C0AD15A486830C08800231A46E92113
S315080059700090FE2002F037F809E0012C07D1192023
S3150800598001230022E9210090FE2002F02CF8F9E21A
S31508005990002C02D14E486830C580FF202D30854244
S315080059A006DA01F03BF80022FE21EA2002F04FF861
S315080059B0E8E251E030E06CE015E002E0D0E0F5E026
S315080059C0AEE0002C0DD14248683000896421484376
S315080059D080B200231A46E2210090FE2002F003F866
S315080059E000E000BFCEE2002C07D164212846FBF771
S315080059F0A7FF81B23648683001813548683000898A
S31508005A00FF21F531884206DC01F008F80022FE2164
S31508005A10E32002F01CF8B5E2002C0DD12C486830C2
S31508005A2040896421484380B200231A46EB2100903E
S31508005A30FE2001F0D8FF0EE0012C0CD12448683076
S31508005A40008A6421484380B201230022EB2100909A
S31508005A50FE2001F0C8FF95E2002C08D164212846F3
S31508005A60FBF76EFF81B21A486830418109E0012CC4
S31508005A7007D164212846FBF763FF81B214486830D2
S31508005A80018200F0CBFF0022FE21EC2001F0DFFFAF
S31508005A9078E2012C2CD10D48B838408803280ADA58
S31508005AA00A48B8384089002805D1012107484173BA
S31508005AB00020074948600022FE21E42001F0C7FFC4
S31508005AC0012102484038417729E000002C040020D3
S31508005AD00C02002098050020F1010020DEFE0000DF
S31508005AE058FE000054FE0000AF01FFFF0002002030
S31508005AF0002C0FD10021F84841774030417300222D
S31508005B00FE21E42001F0A3FF0020F4490870F449BF
S31508005B10486004E00022FE21E42001F098FF31E20B
S31508005B20002C10D1EF48C07A32280DDCED48C17A36
S31508005B30EB486830418200F071FF0022FE21DF2029
S31508005B4001F085FF00E000BF1CE2E5486830408AA6
S31508005B5000231A46DE210090FE2001F044FF11E2E0
S31508005B60002C10D1DF48C07A32281EDCDD48C17A05
S31508005B70DB486830818200F051FF0022FE21E120D7
S31508005B8001F065FF11E0012C0FD1D648C07A322802
S31508005B900BDCD448C17AD2486830C18200F03EFF97
S31508005BA00022FE21E12001F052FFEBE1002C0AD190
S31508005BB0CB486830808A00231A46E0210090FE20F0
S31508005BC001F011FF0BE0012C09D1C5486830C08AE5
S31508005BD001230022E0210090FE2001F004FFD1E11C
S31508005BE0C149BF4868308183C1830184418400F07C
S31508005BF015FF0022FE21512001F029FFC2E1002CE9
S31508005C0010D1002E03D1B448203007830AE0012EB4
S31508005C1003D1B1482030478304E0022E02D1AE48B2
S31508005C2020308783AEE1002C14D1FDF76FFC049079
S31508005C300498000C00231A4653210090FE2001F018
S31508005C40D2FE049880B20123002253210090FE2040
S31508005C5001F0C9FE96E1002C0CD1A1486830C08B32
S31508005C6000909F486830838B00225421FE2001F063
S31508005C7080FE0DE0012C0BD199486830408C0090CD
S31508005C8097486830038C01225421FE2001F071FEEA
S31508005C9078E1002C07D101218F48C1760022022124
S31508005CA09248FEF724FD6DE1002C10D1FF21013149
S31508005CB08C48801DFBF771FE00208A490880022166
S31508005CC08548C1760022FE21562001F0C0FE59E122
S31508005CD0002C16D1002180484030C171002081492E
S31508005CE0088003217C48C176012141774030417301
S31508005CF000207B4948600022FE21572001F0A7FEBC
S31508005D000BE0012C09D100217348C176403041735C
S31508005D100122FE21572001F09AFE33E1002C18D10A
S31508005D2000216D484030C17100206E490880042169
S31508005D306948C17601214177012067494031487396
S31508005D400020674948600022FE21582001F07FFEA6
S31508005D5006E0012C04D100215F48C176403041732A
S31508005D6010E1002C16D100205E49088006215A4809
S31508005D70C176012141774030417300205849486077
S31508005D80B42155482030C1820022FE21652001F049
S31508005D905EFE30E0012C16D100205249088006210B
S31508005DA04D48C176012141774030417300204C4966
S31508005DB04860D22148482030C1820022FE21652051
S31508005DC001F045FE17E0022C15D100204549088050
S31508005DD006214148C17601214177403041730020B0
S31508005DE03F494860F0213C482030C1820022FE210C
S31508005DF0652001F02CFEC5E0002C16D1002039499B
S31508005E00088005213448C176012141774030417325
S31508005E10002033494860B4212F482030C18200222F
S31508005E20FE21662001F013FE30E0012C16D1002079
S31508005E302C49088005212848C17601214177403040
S31508005E404173002026494860D22123482030C18268
S31508005E500022FE21662001F0FAFD17E0022C15D17A
S31508005E6000202049088005211B48C1760121417779
S31508005E704030417300201A494860F0211648203006
S31508005E80C1820022FE21662001F0E1FD7AE00021B0
S31508005E901148C1764030417374E073E072E01449EA
S31508005EA014480068FBF7DDFD0190FCF734F880B272
S31508005EB00F49039010480068FBF7D3FD0190FCF7E3
S31508005EC02AF880B202900398009000229021FE20C2
S31508005ED0029B01F04EFD55E0EC0300200002002075
S31508005EE00C0200209805002004100000003801402C
S31508005EF000007A44900100208C010020002C2ED14D
S31508005F00002E09D12148C7830022FE21522001F024
S31508005F109EFD00F083FD22E0012E09D11B488783F0
S31508005F2000F07CFD0122FE21522001F090FD16E0D2
S31508005F30022E09D11548478400F070FD0222FE2181
S31508005F40522001F084FD0AE0032E08D10F48078489
S31508005F5000F064FD0322FE21522001F078FD11E0D5
S31508005F60002C0DD101200A49487301210848403800
S31508005F70417701200649C8720020044968394860FB
S31508005F8000E000BF00BF07B0F0BD000074020020AB
S31508005F902C040020F0B589B00020089007900690E0
S31508005FA04048007F01287BD13F488079AA2874D1D0
S31508005FB03D48C07932286DDA3B48C079002869DD4A
S31508005FC03949C97908461938FBF758FF08900898DF
S31508005FD0FBF7D4FF0446354A354BFBF76FFE002224
S31508005FE0344B01910090FBF7B7FD039102903248BC
S31508005FF00068FBF7C3FF0646039B029AFBF7C6FE3B
S3150800600005910490FBF7E2FF07902C490798FBF7E8
S3150800601028FD0446FBF77FFF81B22948418308988B
S31508006020FBF7ACFF0646214A214BFBF747FE044621
S315080060300022204BFBF790FD03910290214800684F
S31508006040FBF79CFF01910090039B029AFBF79EFECB
S3150800605005910490FBF7BAFF069018490698FBF7D6
S3150800606000FD0446FBF757FF81B215480183408BB4
S3150800607000901348038B00226021FE2001F079FC72
S315080060800122FE21562001F0E2FC00F0C7FC0021A7
S315080060900448C17600210348C176002101480177EA
S315080060A009B0F0BDEC03002098050020091B9E5E90
S315080060B029CB703F0000F03F8C01002000007A4495
S315080060C074020020900100202A494A88498A511AF8
S315080060D0814209DB274968398968264A683AD162C4
S315080060E00021254A11701BE022494988814217DCA4
S315080060F021490978002913D120490A8F40310A829B
S3150800610001211D4A11701B4968398968194A683A7C
S31508006110D26A891A174A683A5162114689685163E0
S3150800612014498A88898A511A814209DB0021144A4E
S3150800613011701049683989680E4A683A116318E07F
S315080061400C498988814214DC0D490978002910D147
S315080061500A490A8F40314A820121094A11700549C4
S3150800616068398968034A683A126B891A014A683A93
S315080061709162704774020020E4000020CC030020DE
S31508006180E500002070B505460E461446002E02D0DE
S31508006190012E4AD120E0002D02D0012D1AD10CE0A3
S315080061A0602101208007FDF7E1FE0021012080071C
S315080061B0FDF760FF1E4804700CE06021012080078F
S315080061C0FDF7DCFE002101208007FDF75CFF19487A
S315080061D0047000BF00BF28E0002D02D0012D22D197
S315080061E010E013480078A0420BD0602101208007F8
S315080061F0FDF7BCFE214601208007FDF73BFF0C4852
S31508006200047010E00B480078A0420BD060210120F2
S315080062108007FDF7B3FE214601208007FDF733FF0F
S315080062200448047000BF00BF00BF00BF70BD000077
S31508006230A3010020A401002010B5F148407F0128E1
S3150800624074D1EF48C07F0300FEF739FD0805075DE6
S31508006250B0FEFDFCFBFA002010BDEA494868FF21A4
S315080062609131FBF757FB8007800F002809D1802161
S315080062700920C006FCF79BFE0121E348FCF797FEC0
S315080062803AE0E0494868FF219131FBF743FB800774
S31508006290800F012809D180210920C006FCF789FE54
S315080062A00121D948FCF783FE26E0D6494868FF2134
S315080062B09131FBF72FFB8007800F022809D1802137
S315080062C00920C006FCF773FE0121CF48FCF76FFED4
S315080062D012E0CC494868FF219131FBF71BFB800788
S315080062E0800F032808D10121C748FCF762FE8021E8
S315080062F00920C006FCF75BFE10210920C006FCF742
S3150800630056FE0120A8E7BF494868C821FBF702FBEB
S315080063108007800F00280AD180210920C006FCF7D3
S3150800632046FE0121B848FCF742FE38E065E1B5496A
S315080063304868C821FBF7EEFA8007800F012809D1C3
S3150800634080210920C006FCF734FE0121AE48FCF77F
S315080063502EFE24E0AB494868C821FBF7DBFA800724
S31508006360800F022809D180210920C006FCF71FFEEC
S315080063700121A548FCF71BFE11E0A2494868C8217F
S31508006380FBF7C8FA8007800F032808D101219E4829
S31508006390FCF70FFE80210920C006FCF708FE102135
S315080063A00920C006FCF703FE012055E79549486811
S315080063B0C821FBF7AFFA8007800F002809D1802192
S315080063C00920C006FCF7F3FD01218F48FCF7EFFD15
S315080063D03DE08C494868C821FBF79CFA8007800F86
S315080063E0012809D180210920C006FCF7E2FD012118
S315080063F08548FCF7DCFD2AE082494868C821FBF796
S3150800640089FA8007800F022809D180210920C00651
S31508006410FCF7CDFD01217C48FCF7C9FD17E0794959
S315080064204868C821FBF776FA8007800F03280ED143
S3150800643001217548FCF7BDFD80210920C00604E04E
S31508006440DAE0B1E05EE033E008E0FCF7B0FD1021E9
S315080064500920C006FCF7ABFD0120FDE6694948683E
S31508006460FF212D31FBF756FAC007C00F002805D1CA
S3150800647080210920C006FCF79AFD0EE061494868AC
S31508006480FF212D31FBF746FAC007C00F002804D0BC
S3150800649080210920C006FCF78CFD10210920C006C2
S315080064A0FCF785FD01215848FCF781FD0120D3E65C
S315080064B054494868FF219131FBF72CFAC007C00FF1
S315080064C0002805D180210920C006FCF770FD0EE0E2
S315080064D04C494868FF219131FBF71CFAC007C00FE9
S315080064E0002804D080210920C006FCF762FD10218F
S315080064F00920C006FCF75BFD01214348FCF757FD60
S315080065000120A9E63F494868C821FBF703FA800736
S31508006510800F002809D180210920C006FCF747FD15
S3150800652001213948FCF743FD37E036494868C82158
S31508006530FBF7F0F98007800F012809D1802109208F
S31508006540C006FCF736FD01212F48FCF730FD24E094
S315080065502C494868C821FBF7DDF98007800F022817
S3150800656009D180210920C006FCF721FD0121264812
S31508006570FCF71DFD11E023494868C821FBF7CAF955
S315080065808007800F032808D101211F48FCF711FD59
S3150800659080210920C006FCF70AFD10210920C00643
S315080065A0FCF705FD012057E616494868C821FBF7A0
S315080065B0B1F9C007C00F002805D180210920C006FF
S315080065C0FCF7F5FC0DE00F494868C821FBF7A2F96E
S315080065D0C007C00F002804D080210920C006FCF798
S315080065E0E8FC10210920C006FCF7E1FC0121064859
S315080065F0FCF7DDFC01202FE600BF00BF2CE60000FB
S31508006600EC0300200C0200200004004810B5C8481E
S31508006610407B00287ED0C6486038408DFF217D31FA
S31508006620884204DCC2486038008D88421BDDC048B9
S315080066304038C07F002816D1BE494860BE48408809
S315080066400A2810DDBC484088BC4988420BDABA489B
S3150800665080880A2807DDB8488088884203DA03213B
S31508006660B3484038C177B348006CB54988420AD95F
S31508006670AF484038C07F002805D1AE49486003219D
S31508006680AB484038C177AA484078002827D1A8489F
S315080066902038C07801281ED1A648006DA94988422D
S315080066A01DD90020A3490865A1486038C18D008D11
S315080066B081420BDB9E484038C07F00280FD19D4998
S315080066C0486007219A484038C17708E098486038FA
S315080066D0018DC18503E096486038018DC1859448CF
S315080066E0407B012829D1924820380079012820D1F9
S315080066F09048C06C934988421FD900208D49C864C8
S315080067008B486038818D408D81420DDB8848403842
S31508006710C07F00E007E000280FD1864948600721BE
S3150800672083484038C17708E081486038418D8185C3
S3150800673003E07F486038418D81857D484038407F39
S3150800674001287AD17A484038C07F00280BD0002328
S3150800675001221946184601F017FA00231A46194667
S31508006760184601F011FA72484038C07F0300FEF758
S31508006770A6FA08050728486583A1BEDB002010BDD8
S315080067806C484068E121C900884218D90020694947
S31508006790486010210920C006FCF709FC8021092061
S315080067A0C006FCF704FC01216748FCF700FC002141
S315080067B05F4840384177C17701205D490873012059
S315080067C0DDE75C4840686149884218D90020594984
S315080067D0486010210920C006FCF7E9FB8021092042
S315080067E0C006FCF7E4FB01215748FCF7E0FB002153
S315080067F04F4840384177C177012140300173012065
S31508006800BDE74C4840685249884214D90020494996
S31508006810486010210920C006FCF7C9FB8021092021
S31508006820C006FCF7C4FB01214748FCF7C0FB002162
S315080068303F48403841770120A1E776E03D48406867
S315080068407D210901884215D900203A49486010215E
S315080068500920C006FCF7ABFB80210920C006FCF71F
S31508006860A6FB01213848FCF7A2FB00213048403836
S315080068704177C177012082E72E484068E121C900A7
S31508006880884215D900202B49486010210920C006E6
S31508006890FCF78DFB80210920C006FCF788FB012147
S315080068A02948FCF784FB0021214840384177C17705
S315080068B0012064E71F4840682649884215D9002008
S315080068C01C49486010210920C006FCF770FB80218E
S315080068D00920C006FCF76BFB01211B48FCF767FB88
S315080068E00021134840384177C177012047E711480E
S315080068F040681649884215D900200E49486010217B
S315080069000920C006FCF753FB80210920C006FCF7C6
S315080069104EFB01210C48FCF74AFB0021044840388D
S315080069204177C17701202AE700BF00BF27E70000AB
S315080069302C0400200C02002074010020E60F000041
S3150800694070110100B80B000000040048A4060000FE
S31508006950C4090000E40C000010B5052421E08021DC
S315080069602C48FBF71AF880212A48FCF7CFF81221A1
S315080069702848FEF773FB2749898C88420CD125489D
S315080069802838008D2449884204D000F0E9FC00F03C
S3150800699045F800E010BD04E0002000E0401C802817
S315080069A0FCDB2046611ECCB20028D8D100BF0524E6
S315080069B023E080211748FAF7F0FF80211548FCF7F5
S315080069C0C3F812211348FEF749FB1249898C8842FD
S315080069D00ED110482838008D0F49884204D000F09F
S315080069E0BFFC00F01BF802E000F018F8D2E704E05C
S315080069F0002000E0401C8028FCDB2046611ECCB24B
S31508006A000028D6D100BF00F0ABFC00F007F800BFA5
S31508006A10C0E7000074020020FBAA000010B57E2023
S31508006A20FEF7D6F8FCF732F90B490C480185122116
S31508006A302830FEF713FB0949283188848021074846
S31508006A402830FCF7BDF87E20FEF7C2F880210348FF
S31508006A502830FCF7C1F810BDFBAA00004C02002044
S31508006A6070B504460D46E1B20548FDF78BFE00BF3A
S31508006A7001210348FDF729FE0028F9D0204670BDFC
S31508006A8000380140F0B587B0002400200690059034
S31508006A904049088BFBF7FDF907463F49FBF71EF807
S31508006AA005463C49088BFBF7F4F93B490490FBF78C
S31508006AB015F80746394801683846FAF7CEFF0646FC
S31508006AC02946FBF70BF806903549888BFBF7E1F961
S31508006AD006463449FAF7BDFF054629460698FAF7E9
S31508006AE0FDFF059030490598FAF7BBFF0546FBF709
S31508006AF012FA81B22748C183C08B00902548838B40
S31508006B0000225421FE2000F034FF2249088BFBF7AF
S31508006B10C0F920490190C88BFBF7BBF922490090C0
S31508006B20FAF7DCFF07460199FAF79BFF06461A496A
S31508006B30FAF7D4FF17490390088BFBF7AAF907461B
S31508006B401549FAF7CBFF0646144801683046FAF7A6
S31508006B5084FF02900399FAF7C1FF05461149FAF72F
S31508006B6027FF0490FBF7D7F984B20A48C08B0F4970
S31508006B70884204DB0748C08B0D49884204DD02229F
S31508006B80FE21572000F063FF05484038448520461B
S31508006B9007B0F0BD7402002000007A44900100207E
S31508006BA00C0400200000C84100247449B80B0000FA
S31508006BB088130000F0B587B00024002006900590E1
S31508006BC04049488BFBF765F907463F49FAF786FFC0
S31508006BD005463C49488BFBF75CF93B490490FAF7B4
S31508006BE07DFF0746394801683846FAF736FF0646F4
S31508006BF02946FAF773FF06903549088BFBF749F9DA
S31508006C0006463449FAF725FF054629460698FAF74F
S31508006C1065FF059030490598FAF723FF0546FBF707
S31508006C207AF981B227488183C08B00902548838BE7
S31508006C3000225421FE2000F09CFE2249488BFBF7D7
S31508006C4028F920490190C88BFBF723F922490090BF
S31508006C50FAF744FF07460199FAF703FF06461A4969
S31508006C60FAF73CFF17490390488BFBF712F90746DA
S31508006C701549FAF733FF0646144801683046FAF70D
S31508006C80ECFE02900399FAF729FF05461149FAF72F
S31508006C908FFE0490FBF73FF984B20D48403804850F
S31508006CA00848808B0D49884204DB0648808B0C49CE
S31508006CB0884204DD0222FE21572000F0C8FE204645
S31508006CC007B0F0BD7402002000007A448C01002051
S31508006CD00C0400200000C84100247449B80B0000C9
S31508006CE088130000F0B587B00024002006900590B0
S31508006CF04049088BFBF7CDF807463F49FAF7EEFE01
S31508006D0005463C49088BFBF7C4F83B490490FAF75B
S31508006D10E5FE0746394801683846FAF79EFE0646F4
S31508006D202946FAF7DBFE06903549888BFBF7B1F85A
S31508006D3006463449FAF78DFE054629460698FAF7B7
S31508006D40CDFE059030490598FAF78BFE0546FBF708
S31508006D50E2F881B227484184408C00902548038C8C
S31508006D6001225421FE2000F004FE2249088BFBF77D
S31508006D7090F820490190488CFBF78BF8224900903F
S31508006D80FAF7ACFE07460199FAF76BFE06461A496A
S31508006D90FAF7A4FE17490390088BFBF77AF807461B
S31508006DA01549FAF79BFE0646144801683046FAF775
S31508006DB054FE02900399FAF791FE05461149FAF72F
S31508006DC0F7FD0490FBF7A7F884B20A48408C0F49F0
S31508006DD0884204DB0748408C0D49884204DD0222BC
S31508006DE0FE21572000F033FE0548403844852046EA
S31508006DF007B0F0BD7402002000007A44900100201C
S31508006E000C0400200000C84100247449B80B000097
S31508006E1088130000F0B587B000240020069005907E
S31508006E204049488BFBF735F807463F49FAF756FEBF
S31508006E3005463C49488BFBF72CF83B490490FAF782
S31508006E404DFE0746394801683846FAF706FE0646F3
S31508006E502946FAF743FE06903549088BFBF719F8D9
S31508006E6006463449FAF7F5FD054629460698FAF71F
S31508006E7035FE059030490598FAF7F3FD0546FBF708
S31508006E804AF881B227480184408C00902548038C33
S31508006E9001225421FE2000F06CFD2249488BFAF7A6
S31508006EA0F8FF20490190088CFAF7F3FF2249009071
S31508006EB0FAF714FE07460199FAF7D3FD06461A496A
S31508006EC0FAF70CFE17490390488BFAF7E2FF0746D4
S31508006ED01549FAF703FE0646144801683046FAF7DC
S31508006EE0BCFD02900399FAF7F9FD05461149FAF730
S31508006EF05FFD0490FBF70FF884B20A48008C0F492F
S31508006F00884204DB0748008C0D49884204DD0222CA
S31508006F10FE21572000F09BFD054840380485204691
S31508006F2007B0F0BD7402002000007A448C010020EE
S31508006F300C0400200000C84100247449B80B000066
S31508006F408813000070B5044600257E20FDF740FE34
S31508006F50A3480088FA280ADD0020A1490880A1492B
S31508006F600870FF2101319E48801DFAF716FD0121A0
S31508006F709D4881729B4800780300FDF7A0FE08052E
S31508006F802031425BD5FFF1F07E2C11D100209449C7
S31508006F900880012093490870914801880088401CA0
S31508006FA08F4A1080901D445400201146C87002E094
S31508006FB000208B4908800020894908710DE188481E
S31508006FC001880088401C864A1080901D445402207F
S31508006FD08449087010460079001911460871FCE0CA
S31508006FE07F4801880088401C7D4A1080901D4454C3
S31508006FF003207C490870104600790019114608716B
S31508007000EBE0774801880088401C754A1080901D7F
S315080070104454042073490870104600790019114633
S3150800702008710846C470C078002802D105206D4949
S315080070300870D2E06A484079012856D15E2C1CD1E6
S31508007040674800797E30664908717E21644802885F
S315080070500088401C624B1880981D8154801FC07898
S31508007060401EC0B21946C870002802DC05205D49DA
S31508007070087000205A49487155E05D2C1CD15848C3
S3150800708000797D30564908717D2155480288008867
S31508007090401C534B1880981D8154801FC078401E91
S315080070A0C0B21946C870002802DC05204D49087090
S315080070B000204B49487136E049480079001948498B
S315080070C00871084601880088401C454A1080901DB2
S315080070D04454801FC078401EC0B21146C8700028AC
S315080070E021DC05203F4908701DE07D2C03D10120D5
S315080070F03B49487117E03A48007900193849087140
S31508007100084601880088401C354A1080901D445462
S31508007110801FC078401EC0B21146C870002802DC25
S3150800712005203049087058E02D480079C043401CB6
S31508007130C5B27D2D05D15D2C17D1062029490870C9
S3150800714013E07E2D05D15E2C0FD106202549087047
S315080071500BE0A54206D106202249087005E03BE06F
S315080071602BE00BE007201F4908701D48018800889E
S31508007170401C1B4A1080901D44542EE01848018874
S315080071800088401C164A1080901D44547E2C09D154
S315080071900121154840380177002011460880114919
S315080071A0087009E000200E49088000210E48403882
S315080071B0017700200B4908700FE000200949087084
S315080071C0074801880088401C054A1080901D4454D1
S315080071D000201146088000E000BF00BF70BD000017
S315080071E098050020F10100202C04002070B5024605
S315080071F0002013460C461D02FF263602354025435D
S31508007200284670BD86B004460D4626686768A0689D
S315080072100590E06804902069039060690290A0696F
S315080072200190E069009017A0FDF722FD31461BA0EA
S31508007230FDF71EFD39461CA0FDF71AFD1DA0059990
S31508007240FDF716FD1EA00499FDF712FD1FA0039970
S31508007250FDF70EFD20A00299FDF70AFD23A001996E
S31508007260FDF706FD26A00099FDF702FD2948416AAB
S3150800727029A0FDF7FDFC29462BA0FDF7F9FC00BF68
S31508007280FEE700005B48617264206661756C7420D5
S3150800729068616E646C65725D0D0A00005230203DAF
S315080072A02025780D0A0000005231203D2025780D52
S315080072B00A0000005232203D2025780D0A00000001
S315080072C05233203D2025780D0A0000005231322025
S315080072D03D2025780D0A0000537461636B656420B0
S315080072E04C52203D2025780D0A0000005374616336
S315080072F06B6564205043203D2025780D0A00000068
S31508007300537461636B656420505352203D20257881
S315080073100D0A000000ED00E05343425F5348435313
S31508007320523D25780D0A000043757272656E742009
S315080073304C52203D2025780D0A00000006490748D2
S3150800734001850021283041805F218180C18001812B
S315080073500021418170470000FBAA00004C03002071
S3150800736000B5164916480185FF21053128304180A8
S315080073700A210181A021C180CD2181801E21418160
S31508007380AF21C1818C210182BE2181810D490183F2
S315080073900C4925394183052141820A2181820F2121
S315080073A0C18209498183C183018441841221FDF781
S315080073B055FE03492831888400BD0000FBAA000059
S315080073C04C020020782100000410000010B57E2031
S315080073D0FDF7FEFBFEF730FF012800D110BD4F4830
S315080073E0407F012872D14D484030407B002802D0AA
S315080073F001283ED115E040214948FBF7CFFD00287A
S315080074000CD14848406D4849884209D243487838E3
S315080074104089002804D1FDF701FA01E0FDF766FA74
S3150800742078E040494868FF21F531FAF773FAC00752
S31508007430C00F00280ED180210920C006FBF7B9FD30
S3150800744001213748FBF7B5FD10210920C006FBF7D7
S31508007450B0FD0DE080210920C006FBF7A8FD10212C
S315080074600920C006FBF7A3FD01212D48FBF79FFD68
S3150800747050E02A484030407B052828D129494868E9
S31508007480FF21F531FAF746FAC007C00F00280ED1DA
S3150800749080210920C006FBF78CFD01212048FBF757
S315080074A088FD10210920C006FBF783FD31E0802105
S315080074B00920C006FBF77BFD10210920C006FBF753
S315080074C076FD01211648FBF772FD22E023E01348FA
S315080074D04030407B06280ED180210920C006FBF7E4
S315080074E066FD10210920C006FBF761FD01210C4845
S315080074F0FBF75DFD0DE080210920C006FBF759FD6D
S3150800750001210748FBF755FD10210920C006FBF7A6
S3150800751050FD00BF00BF00BF60E70000EC0300207D
S31508007520000400480C02002030750000FCF748FCF7
S31508007530FCF704F8FCF7F4F8FBF740FAFAF7D8FF7B
S315080075400B20FAF707FF0C20FAF704FF0920FAF7D1
S3150800755001FF0320FAF7FEFE01218A48FBF76EF8C1
S315080075604B200002FBF790F901218748417700215B
S31508007570C1770020844940310873C87201218248C6
S3150800758020308170FCF70EF8FCF750FC1A216320B6
S31508007590FCF77AFCFFF7E0F9FCF7FAFF00F08EF942
S315080075A0794878384089002801D1FDF737F97F21D5
S315080075B07E20FDF74BFB00217348C17600207249F7
S315080075C040310871DCE07048C07E0300FDF777FBA8
S315080075D00705134D8B9EB1C4D700FBF757F8FFF785
S315080075E0F5FEFEF775F8FBF7DDFF01F0E3FA7E20FE
S315080075F0FDF7EEFAC3E0002301221946184600F00B
S31508007600C3FA00231A461946184600F0BDFA5F4821
S3150800761040685F49884204D908215E48FBF7C7FCE1
S315080076201DE05A494868FF21F531FAF773F9C00792
S31508007630C00F00280ED180210920C006FBF7B7FC31
S3150800764010210920C006FBF7B2FC01215148FBF7BF
S31508007650AEFC04E010210920C006FBF7AAFCFBF7E4
S31508007660BFF87E20FDF7B4FA89E0FBF70FF8FBF7C1
S3150800767099FF002301221946184600F085FA0023CF
S315080076801A461946184600F07FFA404840684049AD
S31508007690884204D908213F48FBF789FC1DE03B498D
S315080076A04868FF21F531FAF735F9C007C00F0028F9
S315080076B00ED180210920C006FBF779FC102109208C
S315080076C0C006FBF774FC01213248FBF770FC04E0A6
S315080076D010210920C006FBF76CFCFEF75BFC7E2038
S315080076E0FDF776FA4BE0FDF7CDFC20210920C00610
S315080076F0FBF75FFCFAF7CAFFFFF768FEFDF7E8FF3E
S31508007700FBF750FF7E20FDF763FA38E0FDF74EFEE3
S3150800771020210920C006FBF74CFCFAF7B7FFFFF754
S3150800772055FEFDF7D5FFFBF73DFF7E20FDF750FA26
S3150800773025E0FDF7A7FC20210920C006FBF739FC48
S31508007740FAF7A4FFFFF742FEFDF7C2FFFBF72AFF91
S315080077507E20FDF73DFA12E0FDF728FE20210920DC
S31508007760C006FBF726FCFAF791FFFFF72FFEFDF799
S31508007770AFFFFBF717FF7E20FDF72AFA00BF00BF11
S3150800778021E7000000240140EC0300200C02002041
S31508007790204E000000040048FEB546480088FAF767
S315080077A078FB0746444881693846FAF72BFC00D22D
S315080077B0FEBD414A11685068FAF74BF93E498860A0
S315080077C00A46D1689068FAF744F902903A48C168BF
S315080077D001208007FAF745F9009037488168009834
S315080077E0FAF73BF90746344801693846FAF7E0F8EC
S315080077F00446314948690299FAF733F901902E4A45
S3150800780091695069FAF72DF907462B48C169384638
S31508007810FAF764F90546284881682846FAF721F9EF
S315080078200546254A116A5069FAF71BF907462248A0
S3150800783081693846FAF752F9064621463046FAF77C
S3150800784010F9064629460198FAF7B2F8074631466E
S31508007850FAF7AEF8184948622A20085EFAF70EFBCE
S3150800786000901548416A0098FAF7A2F80746FAF711
S3150800787039FB00B2104948852A20085E898D88425E
S3150800788004DD0D48808D00B20B4948850A482A2137
S31508007890415E002902DA0020074948850648C06883
S315080078A00549086108468068C860002001490880C3
S315080078B000BF7DE7500100203C04002010B54021A0
S315080078C00F48FAF76AF840210D48FBF75BF90621DD
S315080078D00B48FDF7C3FB0A49898988420AD108483B
S315080078E02838008D0749884208D0FFF727FDFDF79D
S315080078F08FF903E0FFF722FDFDF78AF910BD0000B6
S3150800790074030020FBAA0000F7B5A0B00C46154684
S3150800791080216846FAF741F8002700267E21684646
S315080079200170FE214170EF2181700721C1702099F5
S3150800793001710021417184712112C1710121017205
S31508007940457229128172012605E06846805DC019D4
S31508007950C7B2701CC6B20B2EF7DBF843401CC1B287
S315080079606846C1727E2101730D21FCF779FE23B0AA
S31508007970F0BDFFB5A1B006461C462A9F802101A886
S31508007980FAF70BF80020009000257E216846017161
S315080079904671229981710721C171239901720021CB
S315080079A0417284722112C17201210173477339121F
S315080079B08173012507E001A8415D00980818C0B247
S315080079C00090681CC5B20B2DF5DB0098C043401C1F
S315080079D0C1B26846C1737E2101740D2101A8FCF766
S315080079E03FFE25B0F0BDFFB585B005460E460E9F95
S315080079F000200190029003900490009000247E21BC
S31508007A0068460171457186710421C1710799017231
S31508007A100899417287723912C172012407E001A8D8
S31508007A20015D00980818C0B20090601CC4B2082C0A
S31508007A30F5DB0098C043401CC1B2684601737E213D
S31508007A4041730A2101A8FCF70BFE09B0F0BDF7B592
S31508007A5084B005460E4600200090019002900390DF
S31508007A60002700247E216846017046708570012132
S31508007A70C170694606980871012405E06846005DEC
S31508007A80C019C7B2601CC4B2052CF7DBF843401C0A
S31508007A90C1B2684641717E2181710721FCF7E0FD7C
S31508007AA007B0F0BD70B504460D467E20FDF790F888
S31508007AB003E02078641CFCF7C3FD2846691E8DB2D6
S31508007AC00028F6D170BD000030B5A1B0044680216B
S31508007AD001A8F9F762FF0025002C02D0012C20D15D
S31508007AE00FE07E21684601710021417144218171B0
S31508007AF01321C1711522104902A8F9F735FF192576
S31508007B0010E07E2168460171FE2141714421817190
S31508007B103321C1713622094902A8F9F725FF3A250A
S31508007B2000E000BF00BF802D03DA294601A8FFF751
S31508007B30B9FF21B030BD0000A6010020BB0100201E
S31508007B40F8B506460C46FAF775FB051E0F4600D033
S31508007B500120014349000B484908411AC90F0DD0B5
S31508007B60002E01D0012100E000210C4361004908E4
S31508007B70401AC00F02D10120FDF7FCF82846394605
S31508007B80F8BD00000000F07F0FB591B000201090FE
S31508007B900F900E900D900C90FA480078642803D048
S31508007BA0F948C07F642803D10121F748017002E033
S31508007BB00021F54801701398002802D001287DD1CC
S31508007BC054E2F248C1891298814203D1EF48C08A2B
S31508007BD00F9001E005200F900F98052802DC05207C
S31508007BE00F9004E00F98322801DB05200F900F99BB
S31508007BF01298411A119881420DDDE348C078002891
S31508007C004FD1E24868384068E0496839C8610121BF
S31508007C10DD48C17045E00F991298411811988142C4
S31508007C203FDCD948C07801283BD1D7482030407876
S31508007C3001282FD1D54868384068D4496839C969B8
S31508007C40401AD34988420DD2CF4898380089462829
S31508007C5020DDCD4898380089801E81B2CA489838F8
S31508007C60018117E0C94868384068C8496839C96950
S31508007C70401A7D21890188420CD9C3489838008961
S31508007C805F2807DAC04898380089801C81B2BE4848
S31508007C90983801810121BC482030417000212038E4
S31508007CA0C170B948C07801287DD1B7482030407BDB
S31508007CB0042806D0B4482030407B00E0FEE30528BF
S31508007CC004D1002201210846FEF75CFA0F991298A2
S31508007CD0411A1198814267DDAC48683840687D21B1
S31508007CE0C900884206D26420A64908700021A64821
S31508007CF08171B4E1A448807900286CD10121A24899
S31508007D008171A248808964285CDA9F484038018DD1
S31508007D10408E081A81B29C4840388186808E099028
S31508007D20FAF7B7F801460A909A480068F9F7D6FEB6
S31508007D300B90FAF723F9984A03C293484038008F04
S31508007D4040430990FAF7ACF80B910A9092480CC890
S31508007D500A98F9F7B3FF904A03C28F4903C9FFF798
S31508007D60EFFE0B910A90FAF731F98C4908608648BC
S31508007D704038008F0890FAF78CF801460990874832
S31508007D800068F9F7ABFE86490A90F9F76AFE0B9088
S31508007D90FAF7C1F8834908700846007864280DDCAC
S31508007DA07C48006801E057E16EE0FAF7E7F8002240
S31508007DB07D4B0B910A90FAF7F5F806D864207949B5
S31508007DC0087002E06420774908706F484038018DD2
S31508007DD04030C18143E16D486838806C7D21C90017
S31508007DE088424CD900206949683988646D4800780A
S31508007DF064283FDA64484038018D4030C0898142A2
S31508007E0033DD0121890763480068F9F7D1FD0B9036
S31508007E10FAF781F881B25C484038028D4030C08953
S31508007E20101A814205DA5F480078801E5D4908709D
S31508007E3020E055484038018D4030C089081A0A901C
S31508007E40FAF71CF80B90534801680B98FAF7DAF81A
S31508007E5010D254480078801C5249087008460078A9
S31508007E60642807DD6420087004E04E480078401D49
S31508007E704C49087044484038018D4030C181494812
S31508007E80007840490870EAE03F48203040780028EA
S31508007E9077D13E488089642803DB64203949087015
S31508007EA0DDE03A48683840687D21C900884206D234
S31508007EB0642034490870002133488171CFE0324884
S31508007EC08079002873D101212F4881712F48808934
S31508007ED064284DDA2C484038018D408E081A81B244
S31508007EE0294840388186808E0990F9F7D2FF0146E5
S31508007EF00A9028480068F9F7F1FD0B90FAF73EF862
S31508007F00254A03C220484038008F40430990F9F7B4
S31508007F10C7FF0B910A9020480CC80A98F9F7CEFEBD
S31508007F201D4A03C21C4903C9FFF70AFE0B910A90B2
S31508007F30FAF74CF81949086013484038008F08903A
S31508007F40F9F7A7FF0146099014480068F9F7C6FD36
S31508007F5013490A90F9F785FD0B90F9F7DCFF1149EB
S31508007F60087008460078642805DD6420087002E079
S31508007F7064200C49087004484038018D4030C1819E
S31508007F806DE063E0F20000200C040020740200207B
S31508007F9070170000D4000020D8000020E000002060
S31508007FA00000C842F10000200000F03FFFE7FE484D
S31508007FB0806C7D21C900884243D90020FA4988642B
S31508007FC0FA48018D4030C089814231DD0121890797
S31508007FD0F7480068F9F7ECFC0B90F9F79CFF81B2BB
S31508007FE0F248028D4030C089101A814205DAF148FC
S31508007FF00078801EEF4908701FE0EC48018D40307C
S31508008000C089081A0A90F9F739FF0B90E848016801
S315080080100B98F9F7F7FF10D2E6480078801CE54977
S31508008020087008460078642807DD6420087004E0B4
S31508008030E0480078401DDF490870DC48018D403073
S31508008040C181DC480078DC49087008E0D748583810
S31508008050007AD949087002E00020D7490870D64846
S31508008060027814991398FEF78DF827E2CF48603006
S31508008070407B012804D002287ED003287DD197E0D2
S31508008080C948683041881298814204D1C648683088
S31508008090408A0F9001E00A200F90C34840687D216E
S315080080A0C900884275D3C14840304079002870D14C
S315080080B0BE48018F4030818201214171808A0A9031
S315080080C0F9F7E7FEBD490B90F9F79CFF19D8B748B1
S315080080D04030808A0790F9F7DCFE01460890B848D8
S315080080E0F9F7FCFCB7490990F9F7BBFCB6490A90C1
S315080080F0F9F75EFC0B90F9F70EFFAC496031087092
S315080081003EE0AA484030808AFF210A3188421ADCBC
S31508008110A6484030808A0790F9F7BBFE01460890CA
S31508008120A648F9F7DBFCA7490990F9F79AFCA6498E
S315080081300A90F9F73DFC0B90F9F7EDFEC1B29B48A2
S31508008140603001701CE099484030808A0790F9F742
S31508008150A0FE014608909948F9F7C0FC9B4909908A
S31508008160F9F77FFC98490A90F9F722FC0B90F9F782
S31508008170D2FE8E49603102E00CE027E009E0087083
S315080081808A4860300078642803DB642087496031B8
S31508008190087029E08448683041881298814204D1E1
S315080081A081486830408A0F9001E00A200F901BE052
S315080081B07D48683081881298814204D17A486830AF
S315080081C0808A0F9001E00A200F900DE0764868300B
S315080081D081881298814204D173486830808A0F904A
S315080081E001E00A200F9000BF00BF0F98052802DCA7
S315080081F005200F9004E00F98322801DB32200F90FB
S315080082006A4860308078002802D11198FDF75CFF33
S315080082100F991298411A1198814219DB62484068F1
S315080082206149086200208863C86360491198C88656
S31508008230084640300079002805D11E215B484030A9
S31508008240817701210171002158484030417042E18F
S315080082500F991298411811988142F8DC534840301A
S315080082600079012809D100215048403001714E4853
S3150800827040684D490862002088634C486030807821
S315080082800028E4D148486830408A0A280BDB46486B
S31508008290406A0A90F9F7FDFD4D490B90F9F71EFC67
S315080082A04C49086020E040486830408A0A2810DABD
S315080082B03D486830408A07280BDD3B48406A0A90EB
S315080082C0F9F7E7FD44490B90F9F708FC41490860BE
S315080082D00AE03548406A0A90F9F7DBFD3F490B90FA
S315080082E0F9F7FCFB3B49086030484030008A0890A3
S315080082F0F9F7CFFD0A902D484030008A0790F9F724
S31508008300C8FD0890334801680898F9F7AAFB099050
S315080083100A99F9F7A6FB0B90F9F730FE304A03C223
S31508008320224860300078401D0590F9F7B9FD09919B
S3150800833008901E484030008A0190F9F7C5FD05915E
S315080083400490274903C9FFF7FBFB03910290059B9D
S31508008350049AF9F71BFD07910690099B089AF9F705
S31508008360ADFC0B910A90F9F7EBFD81B20F4858382E
S3150800837081800D48806A0A90F9F78BFD16490B90A3
S31508008380F9F7ACFB1349086008484030408A089062
S31508008390F9F77FFD0A9005484030408A0790F9F7BB
S315080083A078FD08900B481DE00C020020CC03002045
S315080083B0D4000020F1000020F200002000007A43DB
S315080083C0000082430000BE42000040400000B44264
S315080083D000803B45CC0000200000FA440080BB44E6
S315080083E0E800002001680898F9F73BFB09900A990C
S315080083F0F9F737FB0B90F9F7C1FDF84A03C2F848BD
S315080084000078401D0590F9F74BFD09910890F4484E
S315080084102038408A0190F9F757FD05910490EF49F5
S3150800842003C9FFF78DFB03910290059B049AF9F7A0
S31508008430ADFC07910690099B089AF9F73FFC0B914A
S315080084400A90F9F77DFD81B2E548B838C180FF3852
S3150800845001388089642827DAE24880890890F9F784
S3150800846018FD0A90DF486838406B0590F9F711FD4A
S31508008470DD490690F9F732FB0890DA484188FF3063
S315080084805930008E081A0690F9F7F8FC07900899F3
S31508008490F9F724FB09900A99F9F7E3FAD3490B90FF
S315080084A0F9F71CFBD2490860CD48B838808864289B
S315080084B003DB6421CA48B838818000E0FFE1C84878
S315080084C0B838C088642803DB6421C548B838C18039
S315080084D00120C3498870C2482038007900287DD019
S315080084E001287CD1BE482038807FC2490978884255
S315080084F00DDA0021BA482038817701710020B94980
S315080085006839C8640021B6482038C17764E10F99F4
S315080085101298411A1198814212DDB14820384079E3
S31508008520012804D1AE4801782038C17703E06421D8
S31508008530AB482038C1770121A948203801704BE1A2
S31508008540A748407B0300FCF7BAFB06FD040999FC23
S31508008550FBFDA34801782038C1773CE1A14868387B
S31508008560806BA0496839C96B401A7D21C9008842C9
S3150800857056D99C486838806B9A496839C8639848C0
S315080085806038C18E119881420FDD9548B8388088C9
S315080085900A3081B29248B8388180C08864283BDBAB
S315080085A064218F48B838C18036E00F980B908C4804
S315080085B06038C18E1198411A0B98C20F10184010D6
S315080085C0401C814212DA8648B8388088801C81B2FD
S315080085D08348B8388180C088642801E010E150E1FA
S315080085E01ADB64217E48B838C18015E00F980B90D5
S315080085F07B486038C18E1198411A0B98C20F101823
S315080086004010801C814207DD7548B8388088801E76
S3150800861081B27348B8388180714960391198C88623
S315080086207048683840686F496839096A401A72495B
S31508008630884214DD6A48B8388088401D81B2684887
S31508008640B83881808088642803DB64216448B83898
S3150800865081806448683840686249683908626048B9
S315080086608078002804D15E4801782038C17704E074
S315080086705B48B83801799830C177ACE05948683812
S31508008680806B58496839C96B401A7D21C9008842F0
S3150800869053D954486838806B52496839C86350487A
S315080086A06038C18E119881420FDD4D48B838C088B0
S315080086B00A3081B24A48B838C180C088642838DB95
S315080086C064214748B838C18033E00F980B90444876
S315080086D06038C18E1198411A0B98C20F10184010B5
S315080086E0401C81420FDA3E48B838C088801C81B2E7
S315080086F03B48B838C180C08864281ADB64213848EA
S31508008700B838C18015E00F980B9035486038C18E8F
S315080087101198411A0B98C20F10184010801C8142FC
S3150800872007DD2F48B838C088801E81B22C48B83873
S31508008730C1802B4960391198C8862A48683802E0F2
S3150800874034E023E042E0406826496839096A401A5D
S315080087502A49884214DD2248B838C088401D81B2AB
S315080087601F48B838C180C088642803DB64211C48C8
S31508008770B838C1801B48683840681A4968390862A1
S315080087801748B83881799830C17724E014482038DA
S31508008790C078012805D1002111482038C177817792
S315080087A003E01E210E482038C17700BF0C48203848
S315080087B0C078012805D1002109482038C17781777A
S315080087C003E01E2106482038C17700BF322104483D
S315080087D02038C17700BF00BF58E00000E80000203D
S315080087E02C0400207402002000007A440000C842CD
S315080087F0D4000020F200002088130000581B000057
S315080088003148407B01282AD10F99129841181198AE
S3150800881081421FDB2C48B83801799830C1770F9907
S3150800882012984018801E119988420FDD2748007853
S31508008830002825D12448B8388088401D81B22248AE
S31508008840B838818001202149087019E000201F49A5
S31508008850087015E000211C482038C17710E01A4836
S31508008860407B042803D01848407B052804D1002102
S3150800887015482038C17703E00A2113482038C17704
S3150800888004E0002110482038C17700BF00BF0E4819
S31508008890407B012809D10C482038C07F02460B903E
S315080088A014991398FDF76EFC08E007482038807F76
S315080088B002460B9014991398FDF764FC00BF00BF9D
S315080088C0109815B000BD00002C040020F000002010
S315080088D010B5002201210846FDF754FC4C49088BC7
S315080088E0F9F7D7FA4B490860FEF756FF4848203093
S315080088F0C079002839D14848464948604448008B21
S31508008900B42807D04248008BB32803D04048008BD0
S31508008910B52804D101203E492031487203E00020E1
S315080089203B49203148723D48406E3D49884267D9E7
S315080089303748408B801E3B49098888420DDC3448FD
S31508008940408B801C37490988884206DBFEF732F9D6
S3150800895001202F492031C87103E02D48408B314949
S31508008960088000202D4948664AE029482030C07909
S3150800897001283BD12C48274948602548008BE62822
S3150800898009D02348008BFF212C31884203D0204888
S31508008990008BE72804D101211D482030417203E0ED
S315080089A000201B49203148721C48406E1C498842E9
S315080089B026D91748408B801E1A49098888420DDC3B
S315080089C01348408B801C17490988884206DBFEF746
S315080089D021FA02200E492031C87103E00C48408B69
S315080089E01049088000200D49486609E000200B4917
S315080089F04866084948850122FE215720FFF727F8CF
S31508008A000448408DC2B201210020FDF7BBFB10BD12
S31508008A100C0400203C040020000034430C02002013
S31508008A2088130000000100200000664330B50346A5
S31508008A305A480068181AFF24F534A04201D9574845
S31508008A400360481E904248DD55480078002816D134
S31508008A50881A3C2805DA881A3C24201A514C2070BA
S31508008A6002E000204F4C20704E4800785524201A0A
S31508008A704C4C2070204600784B4C20702AE04B481E
S31508008A800078002822D14A480088401A07280ADDBB
S31508008A90454C2078C40F24186410424D2C70284683
S31508008AA00078414C207042480088401A012808DDA9
S31508008AB03D480078401E3C4C207020460078394CD2
S31508008AC020703B4802800120384C207036480078D8
S31508008AD0344C2070364802805DE0481E90424CDCDB
S31508008AE0481C824249DC2E480078012828D12F48A4
S31508008AF0007800282AD12E480088801A07280BDD1E
S31508008B00294C2078C40F24186410264D2C7028464A
S31508008B100078254C20700DE025480088801A012829
S31508008B2008DB21480078401E1F4C2070204600783C
S31508008B301C4C20701E48028001201C4C207005E049
S31508008B4017480078002801D1164C2070481E90421C
S31508008B5005D115480078401E124C20701BE08A4249
S31508008B6005D111480078001F0E4C207013E00E48FE
S31508008B700078801F0B4C20700DE00020094C2070F7
S31508008B800A4C20700120064C207009480088824251
S31508008B9001DB074802800348007830BD0401002045
S31508008BA0F800002002010020030100200A0100202D
S31508008BB00801002010B5FDF729FD012800D110BDD8
S31508008BC0F848407F00287DD110210920C006FAF711
S31508008BD0EEF980210920C006FAF7E9F90121F248E1
S31508008BE0FAF7E5F90021EF484030417300230122E6
S31508008BF019461846FEF7C8FF00231A4619461846AE
S31508008C00FEF7C2FFE9484068FF21F531884209D2DC
S31508008C10E4484030007B002803D10421E248FAF7F3
S31508008C20C8F9A7E20421E048FAF7C1F90020DD49AE
S31508008C3040310873DD484068DD498842F1D9D94892
S31508008C402030807800281CD120210920C006FAF798
S31508008C50AEF9D64840687D214901884201D2FBF722
S31508008C60A1FD0821D048FAF7A2F90021CD48C1771D
S31508008C700020CC49403148708870CC494862486326
S31508008C801AE04021C848FAF789F9002814D00021CB
S31508008C90C448C1770020C349403148700021C14803
S31508008CA0403081700020C14948624863BD4940315F
S31508008CB048730121BB4841774021BB48FAF76EF952
S31508008CC0002800E011E00BD020210920C006FAF7A1
S31508008CD070F90020B349403148730121B148417702
S31508008CE07D204001B149486044E2AE484030407BAF
S31508008CF00300FBF7E4FF07056DD4FEFDFCFB6C00E3
S31508008D000020A8494031087320210920C006FAF737
S31508008D1050F90020A349403148708870A349486239
S31508008D2048630023012219461846FEF72DFF002343
S31508008D301A4619461846FEF727FF9A482038418DE5
S31508008D400186418D8185018DC185984840687D21C0
S31508008D500901884228D90020964908709148203090
S31508008D608078002802D19149486002E092488F49EC
S31508008D70486040218C48FAF711F900280CD1FBF716
S31508008D8011FD08218848FAF712F97E20FBF720FF23
S31508008D901E20F9F7D1FD02E000208449486004212D
S31508008DA08148FAF704F912E008217F48FAF701F931
S31508008DB07E484068FF21F531884208D979487838D5
S31508008DC04089002803D104217748FAF7F0F8D0E162
S31508008DD076484068FF21F531884204D2042172485A
S31508008DE0FAF7E7F803E004216F48FAF7E0F86F4965
S31508008DF048687D21C900F8F78DFD23282ED26B49D6
S31508008E0048687D21C900F8F785FD192826D96548DF
S31508008E102038018DFF3859384088814207DA614881
S31508008E202038418DFF385938408881420DDB5D482E
S31508008E3040308078012821D100205C4948600862CA
S31508008E40022058494031487318E0002057494860C5
S31508008E50086202215348403041730FE0534948687D
S31508008E607D21C900F8F756FD232807D300204F496E
S31508008E704860086202204B49403148734B4A6832C1
S31508008E805188FF325932508D01231A46FEF77CFE6F
S31508008E9000231A4619461846FEF776FE69E1434846
S31508008EA04068FF21F531884204D204213E48FAF78A
S31508008EB080F803E004213C48FAF779F83B48416812
S31508008EC0683000897D22D2005043814215D2374A44
S31508008ED068325188FF325932508D01231A46FEF7FF
S31508008EE053FE00231A461946184603E01DE1AFE073
S31508008EF064E012E0FEF748FE0EE000212948203023
S31508008F000171002029494860012126482030417016
S31508008F1003202449403148732BE122482038408DEC
S31508008F20FF217D31884204DC1E482038008D8842A6
S31508008F300CDD0023012219461846FEF725FE0023FC
S31508008F401A4619461846FEF71FFE2AE017494868CA
S31508008F507D21C900F8F7DEFC144968314989884241
S31508008F6010D2124A68329188FF325932508D012345
S31508008F701A46FEF709FE00231A4619461846FEF752
S31508008F8003FE0EE007482038018D41860020074978
S31508008F90486000210348203001710420014940310E
S31508008FA04873E6E0EC030020000400480C020020A9
S31508008FB0B80B0000C4000020C40900007048408DAA
S31508008FC0FF217D31884203DC6D48008D88420CDD27
S31508008FD00023012219461846FEF7D6FD00231A4635
S31508008FE019461846FEF7D0FD31E0664948687D21E6
S31508008FF0C900F8F78FFC63496831098A0F39884236
S315080090001ED2604A6832D1895D4A108D012300223A
S31508009010FEF7BAFD5A484030C078012806D1002329
S31508009020012219461846FEF7AFFD10E0554A683288
S31508009030D188534A508D01231A46FEF7A5FD06E04E
S3150800904000205049486005204D496031487390E03A
S315080090504C484068FF21F531884204D204214A4829
S31508009060F9F7A7FF0FE047484068FF21F531884226
S3150800907009D9444840684B21C900884203D20421D3
S315080090804148F9F794FF3F484068404988421ED254
S315080090903C4A6832D1893A4A108D01230022FEF7EC
S315080090A073FD37484030C078012806D100230122D5
S315080090B019461846FEF768FD36E0324A6832D18806
S315080090C02F4A508D01231A46FEF75EFD2CE0042137
S315080090D02D48F9F76EFF2B4840682C49C83188425D
S315080090E022D300202749486025486030C07A0128E5
S315080090F004D1062022496031487305E00021204842
S3150800910060304173403841770023012219461846DA
S31508009110FEF73AFD00231A4619461846FEF734FDAF
S3150800912004211948F9F743FF23E000211448403089
S315080091300171C17013484068154988420CD9FBF77C
S3150800914031FB00200F4948600D48408D822803DC1A
S3150800915001210B4860304173002301221946184645
S31508009160FEF712FD00231A4619461846FEF70CFDAF
S3150800917000BF00BF7E20FBF72BFD00BF1FE50000E8
S31508009180CC0300200C02002000040048A43800008C
S3150800919060EA0000B4910008C800002044010000FD
S315080091A0FC220008049200080C0200209408000023
S315080091B0644D0008015E2D01020304043506070804
S315080091C009ACA24A041A5916011129250A45018132
S315080091D0580B1058594C4C3031313278010B11CBA1
S315080091E07E153E040132050513381206145941321C
S315080091F030303532384834353034324120041B7D1E
S309080092005D7E000081
S705080018C515
